S02C000050443639323030202020202020202020202020203032313132323032313131395F303831365F30303328
S31900001400E826002015D50000FDD1000005D200000000000015
S319000014140000000000000000000000000000000000000000BE
S31900001428000000000DD20000000000000000000015D20000E4
S3190000143C517B00001DD2000025D200002DD2000035D20000DE
S31900001450000000003DD2000045D200004DD20000F59F0000A9
S3190000146455D200005DD2000065D2000019A100006DD20000E8
S3190000147875D200007DD2000085D200008DD2000095D20000A7
S3190000148C9DD20000A5D20000ADD20000B5D20000000000005A
S319000014A000000000BDD20000C5D20000CDD20000D5D20000C6
S319000014B400000000DDD20000E5D200008D9ABDE8FAFAFAFA04
S319000014C834010000C814000027150000C014000000140000D5
S319000014DCFBF30000FCF300002C040000E826002015D50000D1
S319000014F0DCD30000FAD3000000000000FAFAFAFAFAFAFAFA96
S31900001504FAFAFAFAFAFAFAFAFAFAFAFAFAFAFAFAFAFAFAFA45
S31900001518FAFAFAFAFAFAFAFAFAFAFAFAFAFAFAFAC403003121
S3190000152C363A35303A3333000000000000004F637420313881
S31900001540203230313700000000000000F83E490290010A008B
S319000015540100204E323C401FF83E490290010A000100204EB6
S31900001568323C401FF83E490290010A000100204E323C401F44
S3190000157CF83E490290010A000100204E323C401FF83E49027C
S3190000159090010A000100204E323C401FF83E490290010A004E
S319000015A40100204E323C401FF83E490290010A000100204E66
S319000015B8323C401FF83E490290010A000100204E323C401FF4
S319000015CCF83E490290010A000100204E323C401FF83E49022C
S319000015E090010A000100204E323C401FF83E490290010A00FE
S319000015F40100204E323C401FF83E490290010A000100204E16
S31900001608323C401FF83E490290010A000100204E323C401FA3
S3190000161CF83E490290010A000100204E323C401FF83E4902DB
S3190000163090010A000100204E323C401FF83E490290010A00AD
S319000016440100204E323C401FFF0010270A00A40032005000EA
S31900001658A400A4000000000000004A016801E7010000000094
S3190000166C1D0840011D0840011D0840011D0840011D08400166
S319000016801D0840011D0840011D0840011D0840011D08400152
S319000016941D0840011D0840011D0840011D0840011D0840013E
S319000016A81D0840011D0840011D0840011D0840011D0840012A
S319000016BC1D0840011D0840011D0840011D0840011D08400116
S319000016D01D0840011D0840011D0840011D0840011D08400102
S319000016E41D0840011D0840011D0840011D0840011D084001EE
S319000016F81D0840011D0840011D0840011D0840011D084001DA
S3190000170C1D0840011D0840011D0840011D0840011D084001C5
S319000017201D0840011D0840011D08400103203088014E000350
S31900001734A00200FF01FF02FF03FF04FF05FF06FF07FF08FFDE
S3190000174809FF0AFF0BFF0CFF0DFF0EFF0FFF10FF11FF12FF0A
S3190000175C13FF14FF15FF16FF17FF18FF19FF1AFF1BFF1CFF92
S319000017701DFF1EFF1FFF20FF21FF22FF23FF24FF25FF26FF1A
S3190000178427FF28FF29FF2AFF2BFF2CFF2DFF2EFF2FFF0002CF
S3190000179800004C044C044C044C044C044C044C044C044C0467
S319000017AC4C044C044C04555220220000000000004000DC0529
S319000017C06801D002490290013003D30003161300A4004001E1
S319000017D46801E70105053C0098036400000000000000000065
S319000017E800000000000000000000000000001E000E000C01AE
S319000017FC88130B001C000E000A01A00F0B001E000E000A0107
S3190000181088130B001B000E00080188130B001E000E0009010A
S3190000182488130B001C000E000901AC0D0B001E000E000C01D3
S3190000183888130B001E000E000B0188130B005DA1FD5DA1FE1B
S3190000184C5DA2FF5EA3FF5EA3FF5DA2FF5DA1FD5DA1FEBFC010
S31900001860C0C1C1C0BFC00001020203040506070708090A0BA2
S319000018740B0C0700DC057805FF00FFFFFF00FFFFFF00FFFFE7
S31900001888FF00FFFFFF00FFFFFF00FFFFFF00FFFFFF00FFFF55
S3190000189CFF00FFFFFF00FFFFFF00FFFFFF00FFFFFF00FFFF41
S319000018B0FF00FFFFFF00FFFFFF00FFFF3700010378001F0550
S319000018C41F0531051F050100FF01FF02FF03FF04FF05FF067C
S319000018D8FF07FF000000000032008C002C01140000C2EB0B3A
S319000018EC80B5017804290CD0052902D0072904D00BE0401CE0
S3190000190000F00CF802BD401C00F000FB02BD401C01F0A2F82D
S3190000191402BD012002BD0000F1B590B0002569460D84109827
S31900001928447830206043CC4908183230009010980178A54EBB
S3190000193C0127012908D00A2900D131E10B2900D1FFE00E2936
S319000019501CD0252900D11BE1432900D12FE1442900D12AE1E0
S31900001964A82903D0A92900D10AE2AB2900D12FE1AD2900D1DA
S319000019780DE2AF2900D12FE2B02919D0B12900D1BCE18DE233
S3190000198C210009A801F0B3FD09A8C1790691817905914E214D
S319000019A00491039102914179019101790091C37842780178AC
S319000019B4D24874E20021200001F018FD6946C8860321200021
S319000019C801F012FD694688860221200001F00CFD694648868E
S319000019DC0121200001F006FD694608860821200001F000FD47
S319000019F06946C8850921200001F0FAFC694688850A212000A9
S31900001A0401F0F4FC694648850021200001F082FC694608857F
S31900001A180321200001F07CFC6946C8840221200001F076FC66
S31900001A2C694688840721200001F070FC07000B21200001F0FC
S31900001A406BFC06000C21200001F066FC05000098817C2000C5
S31900001A5401F066FA694688770121200001F05AFC6946488475
S31900001A680321200001F0ECFB6946C8760221200001F0E6FB46
S31900001A7C694688760421200001F0E0FB6946487600212000E4
S31900001A9001F0DAFB694608760121200001F0D4FB0590684604
S31900001AA4007E04906846407E03906846807E02906846C07EED
S31900001AB801906846408CC0B200906846837F008D8007800FB4
S31900001ACC6946C98C89000422114001436846808CC000082214
S31900001AE0104008433901102211400143700120221040084302
S31900001AF4AA0140210A4002436846C08EFB2101406846808E28
S31900001B0880000843F72101406846408EC0000843EF210140C7
S31900001B1C6846008E00010843DF2101406846C08D400108435F
S31900001B30BF2101406846808D800108434006400E6946498DDA
S31900001B44C9010143C9B2A448A9E10521200001F04DFC050003
S31900001B580421200001F0DCFB6946888364206843711C884226
S31900001B6C01D2050000E035006846808B642242438A4200D30F
S31900001B80320068468283002392B2A9B2CA48F6E00EAA2000E4
S31900001B9400F0A0FF0EA8818801914E21009143880288C188B9
S31900001BA8C4487AE10421200001F01EFCC1B2C2A007E0062189
S31900001BBC00E00721200001F015FC0100BEA001F099F86EE1B5
S31900001BD0FFFF00000121200001F00AFC8000009949781022B8
S31900001BE411400143032008436946C8750098007888750421C6
S31900001BF8200001F08DFB210001F0AAFF0500009840880028F2
S31900001C0C17D06946888200980079042817DA07AA6846818A86
S31900001C20200001F01BFF00280FD16846818A280001F0C2FFE4
S31900001C340A2808DA6846858A05E00421200001F069FB694697
S31900001C4888820821200001F063FB694688836846808B8001EC
S31900001C5C004901E030F2FF1F09780901974A5118097A89071C
S31900001C70890E0143684681830421200001F0B8FB6946898B21
S31900001C840843694688830521200001F043FB0605360D092154
S31900001C98200001F03DFB0003304306000A21200001F036FB00
S31900001CAC81033143684601830B21200001F02EFB0600012166
S31900001CC0200001F029FB6946098BF2030A4392B204926946C7
S31900001CD4897D03916946C97D02917B49097849080F407F1C54
S31900001CE8FFB20197401CC0B200906846838BDBB2828A2900BD
S31900001CFC77A0D0E070D30000807802A948701098C0786946DA
S31900001D1008721098C279652A01DA160000E0642610988479CD
S31900001D24002C00D001244179002900D00121684601751098E3
S31900001D380079002812D1002721006846007D01F06CFF02003C
S31900001D4C07A80190684600890090330021001098407801F0D1
S31900001D609BFE07E021006846008901F002FF694688830020C5
S31900001D7403003A006846818B5CA000F0BFFF94E00098807EAA
S31900001D88410801220A40074039004F481EE00521200001F03F
S31900001D9C29FB05000421200001F0B8FA694688831420684383
S31900001DB0711C884201D2050000E035006846808B1422424361
S31900001DC48A4200D332006846828392B2A9B2404800F094FFD7
S31900001DD869E000BF88D300000521200001F004FB050004212E
S31900001DEC200001F093FA6946888314206843711C884201D27C
S31900001E00050000E035006846808B142242438A4200D3320069
S31900001E14684682830421200001F0E8FA07000021200001F0B0
S31900001E2877FA69460875200001F0CCFB069090204000A10004
S31900001E3C224A51180818019000880005860F23480090007871
S31900001E50802800D1300000010643200002F03AF80199098816
S31900001E6400018A05940F04434804410F00984078802800D185
S31900001E78080000010143C9B204916846808B0390F6B2029667
S31900001E8CE4B201946846007D0090FBB2AAB26846017E00BF61
S31900001EA015A000F02DFF02E08020694608846846008C11B09F
S31900001EB4F0BD00009CD30000A4D3000025630000257700005D
S31900001EC858FBFF1F3AFDFF1FC8270000C0270000A3FDFF1FA6
S31900001EDC257725772563256325632563256325770000000070
S31900001EF02577256325630000256325772563256325632563E8
S31900001F042577256300000000F1B590B0002069460886B7485D
S31900001F180088C880B6480090B64802903024109F3F78022FD6
S31900001F2C00D197E1042F00D1C4E3052F00D168E3092F00D14E
S31900001F401BE10B2F00D122E10C2F00D18CE11E2F00D157E3AC
S31900001F542B2F00D19EE1312F00D160E2322F00D15AE2332F86
S31900001F6800D16FE23A2F00D112E23D2F00D16BE1472F00D13F
S31900001F7C4BE2482F00D146E2492F00D104E24B2F53D04C2F67
S31900001F9054D04D2F55D04F2F56D0502F57D0562F00D180E171
S31900001FA4592F00D1ACE15A2F00D1A7E1612F00D1F0E0632F98
S31900001FB800D1E6E0842F00D11EE1852F00D1C1E1862F00D148
S31900001FCCBCE1872F5FD0892F00D196E18A2F00D18EE18B2FC6
S31900001FE000D113E28C2F00D10DE28D2F00D107E28E2F00D1A2
S31900001FF401E28F2F00D1FBE1902F29D0912F2AD0922F2BD057
S31900002008932F2CD0942F2DD0952F00D1BCE1962F00D1B7E1E0
S3190000201C982F00D195E1992F00D18DE19C2F00D12EE2A12F19
S3190000203000D1FBE2B02F00D175E2B12F00D16FE2B22F00D12D
S319000020449DE2B32F00D166E2B42F00D161E2B52F00D15BE21F
S31900002058B62F00D155E2B72F00D14FE2B82F00D149E2B92FCE
S3190000206C00D143E2BA2F00D1DEE2BB2F00D15BE3C02F00D131
S319000020806DE3C12F00D1E8E0C32F5FD0C42F6BD07AE3109819
S3190000209444780C2C5BDA200001F015FA08A908706846C088CA
S319000020A80121A140084206D1002008A9487088708C4EFF2080
S319000020BC1DE00B21200002F025F9000108A948700221200004
S319000020D002F01EF908A94978084308A948708870002120008E
S319000020E402F014F986B20321200002F00FF90A2102F02EFB27
S319000020F808A908710621200002F006F908A9C8707948610061
S3190000210C794A5118085A0A2102F01EFB08A948710721200043
S3190000212002F0F6F808A988710821200002F0F0F808A9C8710E
S3190000213408A80E9008200DA908700DAB320021006C4800F03E
S31900002148DBFD1FE3109844780C2C00DB9EE1200002F065FB3B
S3190000215C060002F074FB02003100A2E202F06FFB040002F0F9
S31900002170F2FC02002100C8489BE2C8480088FA21890002F089
S31900002184E7FA81B2E5E28188E3E21098401C00F031FB91E205
S31900002198109840780428D8DA04010822002108A802F0EEFC13
S319000021AC0020009000270225009808A90E180121E0B201F007
S319000021C0ABF83178B84008433070641C04276D1EF3D1009844
S319000021D4401C00900828E9DB08A80E9008200DA908700DAAB6
S319000021E810984178AC4800F087FDCBE2341B002038FDFF1FA5
S319000021FCBEFDFF1FA84CA948807A002804D120684178FD22B4
S319000022100A4042702068A54D002107910691A44909780591EA
S31900002224002104910391029129780191C17800918378427811
S3190000223801789E4800F060FD04220021206802F09FFC002064
S3190000224C28709DE20221002000F05EFD98E200F0D1FD95E224
S3190000226008A800F086FC02E008A800F065FC08A8C0790490E2
S3190000227408A88079039008A84079029008A80079019008A8AF
S31900002288C078009008A8837842780178884874E20098007860
S3190000229C8007800F042101431FE010984178162904D100989D
S319000022B000790407240F15E00724282903D10098007A0440C2
S319000022C40EE0CF0801200C40A0401099C870F0214900074A62
S319000022D8D219515C0840040000D00124210075A036E200BF06
S319000022ECFFFF00004E02000058FBFF1FB0D30000482402E048
S31900002300182400E000240622002108A802F03CFC00200090B0
S319000023140025009808A90F180821E0B200F092FF0600387828
S3190000232869008E4006433E70641C6D1C042DF1DB0098401C73
S3190000233C0090062854DAE7E7482402E0182400E00024062217
S31900002350002108A802F018FC002000900025009808A90F1857
S319000023640621E0B200F06EFF0600387869008E4006433E7065
S31900002378641C6D1C042DF1DB0098401C0090062830DAE7E7BB
S3190000238C482704E0302702E0182700E000270622002108A86C
S319000023A002F0F2FB002000900025009808A90E1800240721B4
S319000023B4F8B200F047FF002800D002240821F8B200F040FF0F
S319000023C8002800D00120317820436A009040084330707F1C16
S319000023DC6D1C042DE6DB0098401C00900628DDDB08A80E90B4
S319000023F00620C0E05C27602415E051275C2412E04627512445
S319000024040FE03B2746240CE030273B2409E0252707E01A2704
S31900002418252404E00B27162401E000270B243D00EDB2A54217
S3190000242C00D39FE030206843C249081844300178280000F019
S3190000244071FDE91B08AA50546D1CEDE7162530206843BB4923
S31900002454081844300178280000F062FD08A949191639087010
S319000024686D1C1A2DEFDB08A8C078039008A8807802900020EB
S3190000247C01900090002308A842780178C2487AE11098447856
S31900002490092C15DBC0487BE1B8D300005AFCFF1FC0D3000017
S319000024A424F2FF1FAC07002054FBFF1F00080020D02700008B
S319000024B8C8D30000256300000B20444327000B37FFB22500F6
S319000024CC05E0FF26E4B2281B08A90E546D1CEDB2BD4207D200
S319000024E00521280000F018FF4608FF2EEFDCEFE708A80E9023
S319000024F4381B3EE05C27602415E051275C2412E04627512495
S319000025080FE03B2746240CE030273B2409E0252707E01A27FF
S3190000251C252404E00B27162401E000270B243D0002E0FF2097
S3190000253030706D1CEDB2A5421AD2E81B08A90E1810980078FC
S31900002544B0380A2807D20521280000F0E3FE052102F0FEF85D
S31900002558EAE70521280000F0DBFEFF28E3DC0521280000F05D
S3190000256CD5FEDFE708A80E90E01B0DA9087088A000F0C0FB72
S3190000258004E1162508A84419163C10980078B22807D10521CA
S31900002594280000F0BFFE052102F0DAF80BE00521280000F045
S319000025A8B7FEFF2804DC0521280000F0B1FE00E0FF202070E1
S319000025BC6D1C1A2DE0DB04210D2001F0A3FE040008A8C078AA
S319000025D0039008A880780290594800784000B049085A0A2145
S319000025E402F0B6F80190554880880A2102F0B0F80090A3B25D
S319000025F808A84278017800BF68A0BEE01098401C00F006FA8D
S3190000260C56E0C07801900298807800904948008B0306DB0F84
S3190000262002984278017800BF62A0AAE00289C18863A03EE093
S319000026345A4810994978002931D057293AD1082210998978F7
S319000026480901C84B59180A3102F0A4FA6846C0890A2102F00B
S3190000265C7BF8694608806846407808A908706846007848704D
S3190000267068464079887068460079C870684680890A2102F0BE
S3190000268467F8694608806846407808A908716946097808AA34
S31900002698517108A94979029165E040886946088068460278F4
S319000026AC417800BF45A000F025FB69E080204000694664E08B
S319000026C0109884780B20444327000B37FFB210984078062802
S319000026D401DBBD485AE0002609E010984178200000F0B0FDA4
S319000026E8F6B208A98855641C761CE4B2BC42F2D308A8807A8D
S319000026FC079008A8407A069008A8007A059008A8C0790490F1
S3190000271008A88079039008A84079029008A80079019008A80E
S31900002724C078009008A883784278017827A026E010984678C2
S319000027380B2E03DBC44827E030F2FF1F042E00DB082683203F
S3190000274C40007100864A5118095ABFA000F0D2FA16E008A865
S3190000276000F024FA08A84079029008A80079019008A8C078B4
S31900002774009008A883784278017800BF19A000F0BDFA01E0DD
S31900002788802008866846008E11B0F0BD002C000001800000B2
S3190000279C25530000B806002025632563257725772577256361
S319000027B02563000025632563256325632563000025772577A7
S319000027C40000000025632563000000002563256325632563CB
S319000027D825632563256325632563256325630000256325631F
S319000027EC256325632563256300000000E0B586B000256A4613
S319000028001582B0490E780278172A4BD01A2A00D18EE0572ACE
S319000028140ED05F2A05D0602A60D0AD2A00D1A5E0CAE08B78DA
S319000028284A78310068A000F067FAC7E0407801001039702908
S3190000283C05D301009039302901D3D02801DB9F48BCE041001B
S31900002850C02802DB9D4A124B04E0802805DBFF22D2439B4BDD
S3190000286459188D5A02E001013F4A555A8006800D3D490E1827
S31900002878307A8007800F0190F0880A2101F066FF0090B7882D
S3190000288C768828000A2101F05FFF81B23B0032004EA08AE09A
S319000028A0C00600208B480578280130490E184E2003906800B7
S319000028B4CB49085A0A2101F04BFF029001954E200090B388CD
S319000028C875881E00814880880A2101F03FFF010033002A0052
S319000028DC41A06AE07C4880880A2101F035FF0290002E03D107
S319000028F006467848408907E07648C0880A2101F029FF0600C2
S31900002904734800890A2101F023FF07007048057801956800FD
S31900002918B249085A0A2101F019FF0090BBB2B2B2029900BF59
S3190000292C31A042E004210D2001F0ECFC86B2002E01D100201B
S319000029400CE0644880880A2101F004FF64214843310001F08C
S3190000295402FF6421484380B201904E2000904E234E22310085
S3190000296825A024E058FBFF1F9D4D0020295E5748007802F081
S3190000297C6FF906000020295E5348007802F0B2F951490F785B
S319000029900021695E0191009030000A2101F0DAFE85B238018F
S319000029A49149085A0A2101F0D3FE82B22B00390015A000F0B3
S319000029B8A3F903E080204000694608826846008A06B0E0BDE2
S319000029CC03800000256325632563000025772577257725637A
S319000029E025630000257725772577256325632577256300004D
S319000029F425772577257725772563000025772563256325639D
S31900002A08257700002563257725772563257700001FB500243C
S31900002A1C0078212810D173480188039101790291817901918D
S31900002A304188009143794E22002100BF74A000F05FF901E0E9
S31900002A4480246400200004B010BD00000480000025770000AF
S31900002A5830B587B00021002402780E2A16D0522A28D104AD45
S31900002A6C6980C178604A128801238B401A4206D02970807838
S31900002A80687004A9042002F03FFA69885AA000F037F914E069
S31900002A94417805A800F02FFD05A84178039181790291417965
S31900002AA801910179009100238278017852A000F023F900E003
S31900002ABC8024200007B030BDA2FDFF1F0180000080FEFFFFDE
S31900002AD0E006002030F2FF1F70B506000D001400082200210F
S31900002AE4200002F04FF804210D2001F00FFCE080062130007A
S31900002AF800F00EFC20281ADA0121300001F07EFC2080002110
S31900002B0C300001F079FCA0800521300000F0FEFB6080252D88
S31900002B2001D1642100E01421484380214902884200D3481EB5
S31900002B34608070BD79B500240025002603E0009804600024DA
S31900002B4800250121300000F04FFC000603D020000124AC40B7
S31900002B5C04436D1C761CF6B2182EECD0302EEEDB00984460F0
S31900002B7073BD79B500240025002603E0009804600024002556
S31900002B840221300000F032FC000603D020000124AC40044375
S31900002B986D1C761CF6B2182EECD0302EEEDB0098446073BDCB
S31900002BACF0B50022124B30270024002556197E439E194436EA
S31900002BC03678062E04DA26000124AC403443E4B26D1C082D39
S31900002BD4F0DB08320470401C302AE9DBF0BD0000C006002061
S31900002BE8B806002058FBFF1FC8170000341B0020257700009A
S31900002BFC30F2FF1F25632563256325632563256325630000C7
S31900002C1025632563256325772563256325770000F8B5040019
S31900002C24BB4862780270817000294BD17F4D0D21200002F005
S31900002C38D0FC002806D12A00290000BF29A000F055F8F1BDF1
S31900002C4CB24E2078B2A7717889070BD5022809D0002805D123
S31900002C60A078072802D1E07855280AD0AC4927E0002806D097
S31900002C7401280ED0022810D0042814D017E0A01C02F0ECFC98
S31900002C88B449884212D10020B3494875F1BDA01C03F0E6FA72
S31900002C9CF4E7A01CFEF724FE0028EFD1F1BDA01C03F064FBCC
S31900002CB0EAE728003178002901D0032915D10100380000F033
S31900002CC417F8F1BD0D21200002F085FC00280AD02078AC280A
S31900002CD807D16078FF2804D10F222100002003F0EDFBF1BD3B
S31900002CEC25772577000000000EB400B501AA0100522004E01D
S31900002D000EB400B501AA0100032000F09DF8009804B000475B
S31900002D14F3B58BB00023079309930893B94800880090002293
S31900002D28012401209040C0B200990500C9B2294203D1079911
S31900002D3C0D43EDB2079574498D182D79254204D0089F060002
S31900002D503E43F6B208966D08254203D0099D2843C0B20990D7
S31900002D64521C082ADFDB0798000600D00223A6480068C078D3
S31900002D784200042002401A430BA80078002801D0FF20087081
S31900002D8C6B4630201856022802D00CA8007888709C4D9D48D0
S31900002DA0008A06900998C0B205900898C0B204900798C0B29A
S31900002DB403902002285C0290487801900020009094480378E2
S31900002DC8002100BF06A0FFF797FFFF20E230285C400920427F
S31900002DDC01D003F0DAFE0DB0F0BD00002563256325632563B7
S31900002DF02563256325632563256325770000000000B585B09B
S31900002E048348817B0491018A0391C17D0291817D0191417D1A
S31900002E180091037DC27C817C04A0FFF76DFF03F0B6FE05B0F2
S31900002E2C00BD0000FFFF0000256325632563256325632563A1
S31900002E402577256300000000F2B588B0050014004E221821B3
S31900002E5401A803F0CDFE684605712D48007801A94870022563
S31900002E68002604E00170761CF6B2761CF6B208988319197894
S31900002E7C002933D0182E31DA6A1CD2B201A84019252902D093
S31900002E9001701500EDE75B78532B0AD0632B02D0772B14D0BD
S31900002EA4E2E7241D211F097801701500DDE72768241D79684E
S31900002EB80029D8D03A78002AD5D001F06BFE38782D18EDB2C0
S31900002ECCCFE7241D211F09886A461180694649780170694653
S31900002EE009784170AD1CF0E70D2101A802F089FB0220084946
S31900002EF40856002801D0012804D10F2201A9C0B203F0DEFA57
S31900002F080020C0430149887009B0F0BD00F2FF1F1905002096
S31900002F1C25770000FAFF000080B50200302A01DB112002BDA9
S31900002F3030235A43374B9A18493293789B0702D500F010F86C
S31900002F4402BD1278D20903D0080000F065F802BD00F0B6F8CA
S31900002F5802BD0000F0FF0000AC070020302250432A4A12185B
S31900002F6C4920135CD80905D0792901D12B2070474720704729
S31900002F80012000291CD0491E1ED0091F1CD01B39012933D90E
S31900002F943139042930D9491F30D00D3924D0C91E032923D9D2
S31900002FA8091F022922D9891F1AD0C91F22D0891E0AD0491E6D
S31900002FBC1CD021E0590901421FD006E05909014208D002E035
S31900002FD05909014201D002207047D808800701D00020704789
S31900002FE401207047492070474A207047482070474B20704779
S31900002FF845207047462070474C20704744207047341B0020D9
S3190000300C24F2FF1F58FBFF1F30F2FF1F55FBFF1F022831D923
S31900003020103802282ED9001F2CD0113830D01D382AD00E3824
S319000030342AD0083802282BD9C01E27D0C01E022828D9C01E5E
S319000030482AD0401E032821D90838022820D9C01E20D0401E62
S3190000305C20D0401E20D0801E20D0401E20D0401E20D0401E94
S3190000307020D0401E20D0C01E12D0401E02D0401E1CD01DE0D1
S319000030842B20704733207047112070473F2070473120704720
S31900003098382070473A20704739207047322070473E207047D0
S319000030AC2D2070472E2070472F2070471A20704747207047EC
S319000030C02C20704730225043924A1218012000296DD0491E1A
S319000030D471D0491E0BD0491E0BD0491E00D1ACE0491E68D0BA
S319000030E80B3960D0491E64D0491E78D0491E00D19FE0491EF2
S319000030FC5DD00C39012972D9891E022923D9C91E79D0491E6E
S3190000311001297AD9891E022979D9C91E73D0491E7BD0491EC1
S319000031247BD0491E65D0133935D0491E5DD00F395DD0491EE9
S319000031385DD0491E79D0491E57D0491E57D0491E57D0491E8F
S3190000314C57D0491E022958D9C91E54D0491E012955D9891E0E
S31900003160022954D9C91E56D0491E03294BD9091F03294AD9C2
S31900003174091F022949D9C91E49D0491E49D0491E012948D99A
S31900003188891E48D0491E48D0491E48D0491E48D0491E48D072
S3190000319C491E26D0891E38D0491E0ED0491E44D049E04932A9
S319000031B011784909014245D00AE049321178490901420CD073
S319000031C404E04921515C4909014201D00220704749321078B4
S319000031D8C008800701D000207047012070472B2070471B20D1
S319000031EC7047122070471C20704725207047242070472620F9
S3190000320070473D2070471F2070471E2070473420704736209D
S31900003214704735207047202070473C207047062070470720CF
S319000032287047082070471A20704743207047452070470320AC
S3190000323C70470420704711207047000038B5302837DA302256
S319000032505043304A14182500383509292FD801A0405C874458
S31900003264084C1C2C3C521222324228782C000021217032BD11
S319000032780321287800F021F8F6E7A8783A34F4E70121A878E7
S3190000328C00F019F8F8E7E8783B34ECE70321E87800F011F829
S319000032A0F8E728793C34E4E70121287900F009F8F8E76878E6
S319000032B43934DCE768793D34D9E7002032BD020008009042D3
S319000032C800D91000704730B50100302048430F4A151845358B
S319000032DC2C78200001236D796D091D4212D1042C0ED1AF4C48
S319000032F090256D0089006118495B0909890708D1F121490026
S31900003304615C8908194200E0072C00D1002030BD30F2FF1FD5
S31900003318F1B582B00346302B03DB062961D15020FEBD302461
S3190000332C6343A04CE31800931D4649351E46263603240C296A
S3190000334053D801A77F5CBF440C141E242A2E363A42588088F6
S31900003354960028784108032043E06846007AFFF7B4FFFEBD0E
S31900003368287841093AE02878810937E0308CFEBD18464E30B3
S3190000337C0088FEBDB07FFEBD307C10282FDA27E0707B2042C9
S3190000339003D128784008204201E00440032C24D111E0317C1E
S319000033A400290CD0491E0CD0491E012907D91E3912D0891E76
S319000033B810D0491E012915D813E00320FEBD0220FEBD307847
S319000033CC04280CD004E0307C022801D0032806D10120FEBD76
S319000033E0A878C10801200840FEBD0020FEBD0000F8B502003C
S319000033F40020302A09DB042901D10320F2BD062901D0072960
S319000034084BD16A48F2BD674B9024640095005D192E195500BC
S3190000341C01240A293FD801A77F5CBF440A10141A2830343E8F
S31900003430646A7400308880060DE031882CE03088810929E005
S3190000344430204243594880184930017822E030880007800F1E
S31900003458F2BD7088F2BDF52040005919081801E05348401948
S3190000346C01786A465170407869460870F3204000185C0009AD
S31900003480204201D14E20087068460088F2BD3088410801E051
S319000034943088C10901200840F2BD3088C00BF2BD80B501001C
S319000034A844A0FFF723FC01E003F0C6FB002003F0E8FB00285E
S319000034BCF8D1404800E000BF401EFCD101BD10B50121012213
S319000034D082403C4B1C8814420CD100205B8813420AD039480F
S319000034E400788008084201D0022010BD042010BD00F01EFDC8
S319000034F810BD38B504000D000020207106212800FFF79EFE5D
S3190000350C217980010843207109212800FFF796FE21794001F7
S319000035200843207108212800FFF78EFE002805D02179C0008B
S31900003534012202430A43227107212800FFF782FE2179400095
S319000035480843207103212800FFF7E2FEE0702079E1788900A0
S3190000355C01432171280000F033F800906846017821700121D2
S319000035702800FFF7D1FE607100212800FFF738FFA0710221D9
S319000035842800FFF733FFE07130206843074908184430017834
S319000035982800FFF7C3FC607006212800FFF7B8FEA07031BD73
S319000035AC58FBFF1F30F2FF1FFFFF00009805002025770000FD
S319000035C07AD40100341B00203DFDFF1F70B582B0060001215C
S319000035D4C0B2FFF70BFF04000821F0B2FFF706FF0500092172
S319000035E8F0B2FFF701FFE107C90F6A0002231A400A438400B7
S319000035FC0420044014430A21F0B2FFF7F3FEC0000821084011
S31900003610204369460870009876BD38B4012100220368001D93
S31900003624002B0BD00468001D0C4202D04D466D1E64192260C0
S31900003638241D1B1FF0D0FAE732BC704710B5002430206043DB
S3190000364C8D490818263004210170302101740021200000F08B
S319000036603EF8641C302CEFDB10BD80B500F007F8854800783E
S31900003674002801D000F063F801BD10B50024302060437F4996
S31900003688081836300178827B202A0DDA032907D0232903D0D9
S3190000369C242905D0302918D1202115E0022113E0222111E030
S319000036B0012907D9891E0CD01E3903D0891E01D00E3908D1B1
S319000036C4232101700121E0B200F007F801E003210170641C9E
S319000036D8302CD2DB10BD10B530225043674A10183230427863
S319000036ECF02313404370002202704378EF241C404470002910
S3190000370000D0828210BD61490978490601D414207047302183
S3190000371448435B4908182630007800280BD0022803D004D3A7
S31900003728032804D007E01220704711207047132070471020B6
S3190000373C7047F020704710B5B3480078400604D5002000F08E
S319000037501BF8002802D0012000F016F80020002130224A4313
S31900003764474B9A182632137C042B03DB537BF0241C4054730E
S3190000377804231370491C3029EEDB4149087010BDF1B59AB047
S3190000378C0120694688700020487001210EA803F0C7F8394878
S319000037A000784000BB490D5A0026002712E0012208216846B3
S319000037B4007800F071FC019833300078FC2101408008044088
S319000037C80C43019833300470761CF6B2684644782000303004
S319000037DC86424DDA302E04DA0EA8805D6946087005E0FFB258
S319000037F002A8C05D694608707F1C68460078FFF782FF8449CC
S31900003804097849060FD5302E0DDA01001139032909D26846B1
S31900003818007802A9085568464078401C69464870D2E7030031
S3190000382C1AA80278A9B26846007800F02BF8ADB2854203DAAF
S31900003840002569468D70C3E72D1A68460078302148430C4955
S31900003854081801903330017803248A080320104003220A4032
S319000038688242B1D01AA909780029ADD003289AD1002299E7DF
S3190000387C684680781BB0F0BD30F2FF1F020800203DFDFF1F52
S31900003890F7B586B01D006846007E30214843BE49081802905E
S319000038A407462837BC7B6846007E03F071FA6946088004263C
S319000038B8202C02D10520B87302E0232C00D1BE73102D07D040
S319000038CC05D3122D69D039D3142D01D039D396E0387F2028F3
S319000038E024DA00216846007EFFF7F9FE2120B8730298493017
S319000038F4019000784007820F08216846007E00F0CBFB019835
S319000039084078064301984670102D01D1202400E02224019843
S3190000391C00788106C90F6846007E00F013FA0AE001216846D7
S31900003930007EFFF7D4FE102D01D1232400E0242400206946EA
S31900003944088060E0387F20282EDA3888B8816A463988684682
S31900003958007E00F07FF86846808B6946098888420BD28C48FC
S3190000396C0078C0094BD0F88B6946898B884202D20846694604
S31900003980088008A8007800283FD068460088F883112D01D185
S31900003994002438E0387F202801DA022433E0032431E0387FDB
S319000039A8202808DB032C2CD1232401216846007EFFF791FE94
S319000039BC25E003A96846007E00F028F80425680003A9095A64
S319000039D000291AD0B9816A466846007E00F03EF802280ED086
S319000039E4684600886946898B884208D208A80078002808D004
S319000039F868460088F883012403E06D1E6DB2002DDFD5BC7342
S31900003A0C6846008809B0F0BD39FDFF1F70B5002200235E4E9A
S31900003A205C003025454375192D192D8D0D535B1C052BF5DBEE
S31900003A34501C030052008A1808E014885D004D192E88A64230
S31900003A4801D216802C805B1C052BF4DB0200052AECDB70BDB4
S31900003A5CF7B504000D00302060434C490F1832370126F87DDF
S31900003A7041093140200000F0A9F80299019100953B78020059
S31900003A84F87D400906403100200000F003F8FEBDC006002047
S31900003A98F7B582B018000021002500246A461170002802D188
S31900003AAC6846008D3FE03B494843642100F04FFE39494618F5
S31900003AC06846007B002800D076086846008D70438000354961
S31900003AD4884221D20195344F344D01987043642100F039FE89
S31900003AE8281A390000F035FE01006846008D784300F02FFE12
S31900003AFC0500641C0198854202D0E4B20A2CE5DBFA20400013
S31900003B1045432800390000F020FE0AE06846007A30214843B6
S31900003B241C4908184630008802216A4611706946098A80B23C
S31900003B38814207D2084669460978002902D101216A4611700A
S31900003B4C0B9908806846007805B0F0BD80B5302251430E4A38
S31900003B60511832310A78CB7D9906C90F00F001F802BD10B5D1
S31900003B7404000223002A0CD0002900D0032360430C3292B2C4
S31900003B88DA405043094900F0E4FD201A80B210BD30F2FF1FDA
S31900003B9C40FDFF1FD4300000DC05000040787D011027000062
S31900003BB0404B4C0050C30000814201D2401A02E0C2435018D2
S31900003BC4401C80B27047000038B5A44CA44AA35C0322802B08
S31900003BD807D190235B0085006419E35A9C0A0323234030242B
S31900003BEC6043B24C24183334032B02D1E07D800903E0A07D94
S31900003C00430803201840E378102B07DA207880080240032ADE
S31900003C1401D1002000E0012000F001F832BD0200A54B03D006
S31900003C2802280BD002D30AE0188808E0A2480078C00701D537
S31900003C3C988802E0588800E0D888002900D0400080B270472A
S31900003C50F1B582B06846007A30214143964A51184631009134
S31900003C640D887E4F9021490080003818465A01243106890F86
S31900003C7821406846007AFFF7A5FF7849795C802901D13105C8
S31900003C8C890F02292BD0A84200DA05008A4881888D420DDA06
S31900003CA041888D4201DA007800E040782E0045432800642124
S31900003CB400F04EFD3518ADB200984079009909898D420CD2E6
S31900003CC88108214206D00A2203216846007A00F0E1F9F7BD2A
S31900003CDC0421014301E0FB21014000984171F7BDF8B5002656
S31900003CF00024714F302060433D183635A87B202815DA287829
S31900003D04102812DB0121287D800808420DD0E87C400901401C
S31900003D18E0B200F019F82882E0B200F0A1F8287DFB21014037
S31900003D2C2975641C302CDFDB302070433818443000782028C2
S31900003D4002DAF0B2FFF784FF761C302EF2DBF1BDF2B582B02E
S31900003D5406005C4990225200B300CB189A1800923F4A895C5E
S31900003D680327802907D16946009A1288920A032313400B7122
S31900003D7C01E06A4611716946097AFFF721FF040068460079A7
S31900003D90002805D0022831D007D3032805D03AE0009840889D
S31900003DA4844226D234E0302046434248801945300578072D11
S31900003DB801D0052D01D1002511E00079400807403A00684616
S31900003DCC017A280000F023F8002F02D0042D00DA20002500DE
S31900003DE0844200D9050068460079032813D100984088A842A5
S31900003DF40FD3009845880CE000980088000607D517206043A6
S31900003E0880B2142100F0A2FC050000E02500A8B2FEBD18B5BF
S31900003E1C2A4C042812D18B235B00E318012A02D0022A09D001
S31900003E300AE0F3204000205CC00701D5588808E0188806E0D4
S31900003E44988804E083235B0040002018C05A002902D0002AA8
S31900003E5800D0400080B212BD58FBFF1F4B02000010B5174A5B
S31900003E6C1749535C0100802B06D190235B008C001219D25AB9
S31900003E801205930F032B16D1302251430A4A511846310A79BD
S31900003E949206920E0D4B1B780C88A34203D2402313430B716E
S31900003EA800E00A7109798A09082100F0F3F810BD30F2FF1F7F
S31900003EBCD01700003EFDFF1FD817000058FBFF1F4B020000FF
S31900003ED0DE1700003E4A3F49535C802B07D190214900800027
S31900003EE41018405A8005800F7047002B1ED030225043384AB7
S31900003EF8101836300278102A10DB052B14D0C07B002805D037
S31900003F0C401E022806D9C01E08D005E0032B09D0012B07D08F
S31900003F20062B05D001207047022B01D0012BF9D100207047DE
S31900003F34F8B50400284F3878002845D00921200000F0E4F947
S31900003F4806000A21200000F0DFF9050004210D2000F0DAF92C
S31900003F5C20490978B6B2721880B2824201DA0920F2BDADB267
S31900003F70AE4205D2A81B80B2814201D20820F2BDB86A61008B
S31900003F84C8408007800F05D0022807D004D3032806D019E05E
S31900003F980520F2BD0620F2BD0720F2BD0021200000F09EFDC4
S31900003FAC01280BD00121200000F098FD012805D002212000EF
S31900003FC000F092FD012801D10A20F2BD0120F2BD58FBFF1F53
S31900003FD44A02000030F2FF1F5C070020E618000080B5090286
S31900003FE80143684601806946052000F089FF01BD80B5090202
S31900003FFC0143684601806946072000F07FFF01BD80B58F234F
S319000040100340080118434006400ED101014368460170694677
S31900004024102000F06FFF01BDF0B5017830292EDAF52252004E
S319000040384900AF4B591889180B7883704A780271FF2B22D052
S3190000404CAB49AC4CCB181B5D1C0944700C2C1ADA8379A94D1C
S319000040604D190126002B03D02F88E740374210D000244471AB
S31900004074FF2A0FD0A14C8918095D0909C1700C2905DA002BB4
S3190000408805D02A88CA40324201D10020F0BD46710120F0BDF5
S3190000409CF2B58EB01700FD2600256C4680286BD1002939D0FE
S319000040B0012961D0032902D004290FD01AE1302068439149C1
S319000040C408184C21415C31404C3001706D1C302DF3DB39006D
S319000040D880209BE08848874949190A1810780109884B1B8887
S319000040ECCB40DB0714D50207920E03096C2463437F4CE31833
S319000041009A1880320007800E6C2359436118081880300068D0
S319000041140121B940884310606D1C602DCCDADBE76022FF211B
S31900004128B34800F02DFD012102A802F0FBFB302602A880191B
S3190000413C401E007820700120A0716846FFF770FF002810D0B6
S31900004150A07897210901EDB2684A521950546D1C6079002891
S3190000416405D02079EDB2644A521950546D1C761E05D0DFE7BF
S31900004178C02200219F4800F003FDB7E00EA909780200813AC7
S3190000418C0D2A03D20329F6D139003DE020700120A0710329D6
S319000041A000D1A5716846FFF741FF0028E9D00EA80078801E8D
S319000041B40728E4D801A1095C49008F440317992C3C41728095
S319000041C8A07840008B4909180120B8400A8802430A8061793C
S319000041DC002906D021794900854A51180A881043088081E0E1
S319000041F0207830214843444908184930C1780E40C670390025
S31900004204A078FFF7EDFE6079002871D039002079FFF7E6FEB9
S319000042186CE0207830214843394908184930C1780E40C670F4
S3190000422C3900A078FFF7E2FE607900285CD039002079FFF75C
S31900004240DBFE57E02078302148432F49081849300178BF2275
S319000042540A40B901402319401143017067482749A278254B22
S319000042689A18515C0907090F6278D2008218575461790029C1
S3190000427C3AD0217830225143204A511849310978890631D53C
S319000042901B4922799A18515C0907090FE278D200801847542F
S319000042A426E03A00A178607800F02EFA607900281ED03A008E
S319000042B82179E07800F026FA18E03A000E48A1780C4B591881
S319000042CC085C0107090F6078FFF79AFE607900280AD03A00D9
S319000042E007482179054B5918085C0107090FE078FFF78CFEBE
S319000042F40FB0F0BD58FBFF1F501500206C050000E4050000F4
S3190000430830F2FF1F361B0020F2B583B0010000220020B24BD0
S3190000431CB24C4D006D185D192C196C254D435D19503501954A
S3190000433006250E006E439D190095AC4D5D1902952E8801255C
S319000043448D403540FF2156316E46367B0A2E4ED801A7BF5DEF
S31900004358BF4400BF0C1624324E565C66707A8400002D42D0FE
S3190000436C009800883FE0002D3DD0009880788007800F38E000
S31900004380002D36D0009880788006000F31E0002D2FD00198F5
S31900004394418896484843BB30BB21490000F0DBF99349401AD3
S319000043A823E0AB20C0001A5A1AE0029800791CE0002D1AD0D9
S319000043BCA078A27017E0002D15D02078227012E0002D10D08B
S319000043D0607862700DE0002D0BD00198028803E0002D06D02B
S319000043E401988288C8205043AA3000F0B4F900B204B0F0BD17
S319000043F8C01E0020EC020020CC010020F2B584B0070001AC23
S3190000440C27700125A57100266846007C092800D1A67101A8B1
S31900004420FFF704FE00285DD030204743B348C019483000907F
S319000044340F216B4AB14B6846007C092800D9CBE001A73F5C6B
S319000044487F00BF44043A5D5F6872B9B1B9A5A078AA4B101807
S3190000445CC3181B780F20184040001B096C267343D31818188A
S319000044706E300388607900281BD02679A14894192618307802
S319000044840140490000096C246043101840186E300088009919
S3190000449849784909294203D01818C3031B0C04E0009909789E
S319000044ACC90900D10300C8205843AA30FF21563100F04DF916
S319000044C020E0A0788F4B1018C31818780F2303405B00000984
S319000044D46C2568431018C0185E3000886379002B7BD026798B
S319000044E8864B9419E6183378194049001B096C246343D218AD
S319000044FC51185E310988401880B26AE0012068E060786C217B
S3190000451048431018B1300078400805403AE0607900285CD0B1
S31900004524009840788106C90F0120484055E0A078734B1018F2
S31900004538C31860786C26704310181E780E408619A936367839
S3190000454C002E01D0012006E04A30068801201B780B40984070
S3190000456030406379002B3AD02679664B9619F618E3786C24C8
S319000045746343D21833780B40D318A9331B78002B05D14A32D0
S319000045881288337819408D4015400543280022E061780120ED
S3190000459C884080B2617900291BD0E1788D400543A8B216E05F
S319000045B06079002807D1A078185C0102872007E060790028FA
S319000045C406D0A078185C00022179595C084304E0A078185C6F
S319000045D8000200E0002005B0F0BD000050150020DD090000FA
S319000045ECE4050000521C0000D20A0000F0B583B06C46207068
S319000046000120A0716846FFF711FD002874D03E483C49A2782B
S319000046148218525C0F210F2313409B0012096C256A43821801
S31900004628D2188032176800226379002B37D0334B25794519B3
S3190000463CEB181D780F262E40B600B4462E096C256E43851962
S319000046506646AD1980352D683D432F001D780F232B409B0018
S319000046642D096C2675434519EB1880331A70244B25794519B3
S31900004678ED5C0F232B409B002D0975434519EB1881331A701A
S3190000468C1D4B25794519ED5C0F232B409B002D0975434519E3
S319000046A0EB1882331A70174BA5784519ED5C0F232B409B0060
S319000046B42D096C2675434519EB1880331A70104BA5784519F8
S319000046C8ED5C0F232B409B002D0975434519EB1881331A70CA
S319000046DC094BA4780419E35C194089001B096C246343C018E4
S319000046F04018823002703800FEBD000030F2FF1F8C02002053
S319000047046C0500005015002080B5000208430005000D1103FD
S3190000471801436846018069460F2000F0F1FB01BDF44600283A
S3190000472C04D4494200F013F8404260474042002905D45FD039
S3190000474000F00BF8404249426047494200F005F8494260470E
S3190000475403460B43E6D40022030A8B420BD203098B4219D25D
S3190000476843088B422ED2411A00D20146524110467047FF22EA
S3190000477C09023FD012068B4205D3121209028B4201D3121258
S31900004790090203098B4219D300E0090AC3098B4201D3CB0113
S319000047A4C01A524183098B4201D38B01C01A524143098B424F
S319000047B801D34B01C01A524103098B4201D30B01C01A524134
S319000047CCC3088B4201D3CB00C01A524183088B4201D38B0078
S319000047E0C01A524143088B4201D34B00C01A5241884200D311
S319000047F4401A5241CFD201461046704708B502F035FB08BD25
S3190000480810B5974C2C21200002F010FA9548A06200F044F979
S3190000481C002801D100F034F810BD70B505000026002004002B
S319000048303100280000F058F90100700081402143C8B2761C32
S31900004844032EF2DB70BD58B5002400F029F9002801D10120D1
S3190000485852BD00F07CF9FA218900884201DB022052BD002631
S3190000486C3100200000F03AF9032808D0761CF6B2032EF5DB80
S31900004880641CE4B20C2CF0DB002052BD80B5002802D000F0B7
S3190000489460F9401C80B200F03BF901BDF8B504006C20604361
S319000048A871490D185035FF2656362988C8204843AA303100B2
S319000048BCFFF74DFF87B2A988C8204843AA303100FFF745FF7E
S319000048D080B2874225DB3D1AADB266488188A94201DA02207E
S319000048E4F2BD4188A94201DA0120F2BD0088A84213DB00212B
S319000048F8200000F0F5F801280BD00121200000F0EFF8012863
S3190000490C05D00221200000F0E9F8012803D1152D01DB00206D
S31900004920F2BD0320F2BD38B500250024280000F019F8690034
S319000049348840204304006D1C0C2DF5DB4948846200F001F848
S3190000494831BD47480178002907D14178042902DA491C417086
S3190000495C704701210170704770B582B004000320694608709B
S31900004970414800880121A140084226D02000FFF78FFF06002F
S3190000498400256000001937490818401981784900AE4203D17C
S3190000499801220A43827000E08170807800F014F800280BD0DB
S319000049AC684606703100200000F098F8002803D131002000AF
S319000049C000F084F86D1C032DDDDB6846007876BD10B50021C1
S319000049D400224006400E03000B41DC07E40F1219D2B2491CDA
S319000049E80729F6DB042A01DA002010BD012010BDF0B583B0F8
S319000049FC00241A4F6D46302060431D490E1844363078142884
S31900004A1026DBF079F7210140F17101201849097849080142D0
S31900004A241CD02C70A8716846FFF7FEFA002815D0B96A0320E8
S31900004A386A7852000B00D3400340032B08D16A79002A09D0E2
S31900004A4CEA785200D1400840032803D0F07908210143F1710D
S31900004A60641C302CCDDBF7BD5C070020FFFFFF0050150020FF
S31900004A74E0180000341B002030F2FF1F41FDFF1F08B4024B1C
S31900004A889C4608BC6047C04627F0FF1F08B4024B9C4608BCDD
S31900004A9C6047C046BDF0FF1F10B52E4C1422216831A002F0C7
S31900004AB0E0F9000605D1606800680021C943884201D100201E
S31900004AC410BD012010BD000080B58A0025A189580C235843ED
S31900004AD8214B1B68181880181830FFF7D7FF01BD89000C2284
S31900004AEC50431C4A12681018401880691BA25158884201D1D2
S31900004B00012070470021C943884201D1002070470320704749
S31900004B14F1B51348FFF7B4FF104E3468002500BF13A707E05E
S31900004B28EDB2A80039582000FFF7B0FF6D1C241D3068010073
S31900004B3C14318C42F2D3694609881430FFF7A4FF0121706870
S31900004B50FFF7A0FFF1BD02480068406980B270471CF2FF1F98
S31900004B6400900100110000002200000033000000564F505FEC
S31900004B785F5F534543544F525F5F5F56414C494410B504003F
S31900004B8C10000A000100200002F01EF8200010BD124207D0B4
S31900004BA08B0706D00B78491C0370401C521EF7D8704783075C
S31900004BB406D00B78491C0370401C521EF9D1704770B4103AFB
S31900004BC803D378C9103A78C0FBD2530701D318C918C001D5B0
S31900004BDC08C908C0D20704D30B880380891C801C002A01D51F
S31900004BF00B78037070BC704770B500F0B0F800F0B4F85F48D2
S31900004C04007840070CD500245D4E5E4D0020295E200000F0C5
S31900004C1821F861007052641C102CF5DB70BD80B52022584975
S31900004C2C5548FFF7B5FF01BDF0B55349554A127852008A180B
S31900004C4013880024534D2601AE5B6700CE53641C102CF8DBB4
S31900004C54002800D11380F0BDF0B585B00C004C4900010D186C
S31900004C68F32040000F18012638788008304201D1288837E04E
S31900004C7C102229006846FFF78BFF297B0A2041433878C708C4
S31900004C90A1421EDA601AEA8950436A7B0A235343591AFFF79E
S31900004CA45AFD01B26846C08981420CDA68464089401A6946CC
S31900004CB8488137420FD0098880B2884209D2084607E0002004
S31900004CCC6946488105E0374203D068464089694608806846C9
S31900004CE0408969460988884200D3084605B0F0BD284AF323DC
S31900004CF45B00D35C5B0706D500011018027B0A235A4391429C
S31900004D0801DA01207047427B0A205043814201DA02207047ED
S31900004D1CC830814201DA032070470420704780B5172002F0D4
S31900004D30FCF88008B2218900884209DB2821484380B21B21A1
S31900004D44FFF706FD96218900401A04E00101081A0004000DA9
S31900004D58E13800B202BD80B5FFF7E3FF0849888001BD074844
S31900004D6C0421415E0222825E084B9A4200D01100018070471D
S31900004D803EFDFF1FC0060020B8060020E006002030F2FF1FB6
S31900004D9458FBFF1FFF7F0000F0B585B000259D49097808297F
S31900004DA801D1012400E000249A4F9B49791802919A49791891
S31900004DBC0191012846D0994A00213800FFF7DEFE06220021B5
S31900004DD003A8FFF7D9FE01009448381800909448009A1061AD
S31900004DE403AE002C12D0012002F0C4F830889049098888423B
S31900004DF807D17088002802D1B088002808D0062000E00A206E
S31900004E0C8249087003A9002002F0B0F8308800990880009872
S31900004E20008800994880002C02D10C2002F07AF9C020C0005F
S31900004E343B1864220821019802F084FA922000013B1805222C
S31900004E480821029802F07CFA019802F092FA029802F08FFAF9
S31900004E5C012000F027F80C22FF218C48FFF78EFEA82200217D
S31900004E708A48FFF789FE602200218948FFF784FE88490D808F
S31900004E8488490D70202200218748FFF77BFE87490D70874908
S31900004E980D70874845810020C043B14908600220B049785482
S31900004EAC05B0F0BD38B50400784D6022002128006C30FFF777
S31900004EC063FE60220021CC352800FFF75DFE534D0A2200216D
S31900004ED4A6482818FFF756FEA4482818FF2101708170032279
S31900004EE80379134003714171C171417A0A404272002C04D0D0
S31900004EFC60220021C148FFF741FE31BD7CB502006B461A705F
S31900004F10424C0F20122A1AD801A5AD5CAF4400BF16161438C3
S31900004F2440481676167654606A767C849E163000019169461A
S31900004F383A48201802F02DFA002804D1B148817802220A432C
S31900004F4C827073BD087800F035FA73BD080002F0A6FA73BD90
S31900004F60080002F0A9FA73BD0D88290AE8B202F0ABFA73BD41
S31900004F741822A648201802F0BBFBDAE70020C043784908600E
S31900004F8873BDA2482018027810251543057008889880CCE7E6
S31900004F9C0C229D200001E9E70D8801232A0BC749EEB2A419E4
S31900004FB0615C01402C0A204002F0A2FB73BD0B78DA095906CF
S31900004FC4490F184002F08AFC73BD1CB56A461070114A8F4B45
S31900004FD8D318002803D0022807D003D30AE01878FD2404E083
S31900004FEC1878FB2401E01878F72404401C700191694608480F
S31900005000101802F0CAF9002804D18048817804220A43827096
S3190000501413BD000054FBFF1F501500205C090000480900000A
S31900005028040A0000E40500002C020020BE240020F4B5060078
S3190000503C0C0002F08CFD0700B04D3100B04802F0D2F90028C1
S3190000505019D1E86805210180083002F003FE54216854685C45
S31900005064002804D102211035280002F005FE0099380002F0ED
S319000050787CFD0028E3D063488178082205E03078844204D0D5
S3190000508C5F48817810220A438270F1BDC0010020AC0300209B
S319000050A0CC010020FA070020F80700208C0700208807002067
S319000050B48907002030F2FF1F1CB5AC4C6946AC48201802F05C
S319000050C894F969468888514AA4180978002910D0012917D090
S319000050DC02291ED006292BD007292CD009292FD00C2930D0E5
S319000050F00D2935D011291CD013BD02F07FFD20780221014308
S31900005104217002F0C9FD13BD02F076FD207804210143217081
S3190000511803F0F2F813BD02F06DFD2078082101432170019845
S3190000512C03F010FB13BD02F063FD02F0F2FB13BD03F0ACFA01
S3190000514013BD010AC0B203F0B7FA13BDA249088013BD00F061
S31900005154DDF82078EF210140217013BD00F0B4F813BD0000B6
S31900005168F4070020DC090000E9050000F8B50123012100202C
S3190000517C7C4A6C278410640F2418E410E5B2944E755DE4005A
S31900005190061B0124B44025422CD04B4C15182D192C7824098D
S319000051A48E4E965BE6401E4222D02D782E07360F7C431419A1
S319000051B84A342488F4401C4218D174002D096C2675435519D6
S319000051CC2C196E342488844DAC420DD30B4909180C78641C1E
S319000051E00C70E4B2022C04D10D2102F06DF90220F2BD002128
S319000051F4401CC0B26028C1DB002901D00020F2BD0120F2BD16
S3190000520858060020E4240020CC050000010A0000F8B5040059
S3190000521C012501266B4601229C2103F0DBFD6846008802286F
S3190000523047D06B4601229C21200003F0D1FD6846008802287B
S319000052443DD06B4601229E21200003F0C7FD0426464F68466C
S31900005258008806216143795A88421DD16B4601229D212000AC
S3190000526C03F0B8FD68460088002813D05B4861000919791888
S31900005280081869460988314205D04178FF2907D0491C41709E
S3190000529404E00178FF2901D0491C01704F4839180A88012039
S319000052A8A04082430A80B748006881780E438670B548817820
S319000052BC0D43857000263000F2BD00006C050000DCB5070085
S319000052D0002600240120A040074204D0AD4AA821200003F089
S319000052E469FD641C0C2CF3DB0A2002F096FC0120B0400742BC
S319000052F802D0300001F012FF761C0C2EF5DBD3BDB804002090
S3190000530CAC1E002030B583B0040000250120A840A1B20142BD
S3190000532011D002229C21280003F046FD6B4601229C2128009A
S3190000533403F054FD68460088022802D00120A84084436D1C90
S319000053480C2DE5DBA4B2002C06D02000FFF7BAFF8F480188CB
S3190000535C0C43048037BD80B501F0FAFD80208C49086001BDB8
S31900005370501500204809000080B500210C2002F08DF801BD96
S3190000538480B501000A001448802A04D10C22FF21FFF7F8FBBD
S3190000539801BD0B00813B0D2B04D2FF2180188138017001BDC8
S319000053ACD2088018027801234907490F8B401343037001BDDD
S319000053C0C108064A51180A7801234007400F83409A430A70FB
S319000053D470470000FA070020C0010020E40500008902000092
S319000053E8DD090000FEB56C4FF868083002F036FC542178545A
S319000053FC785C002800D1C2E002210C2002F048F802F0D1FAEA
S319000054106448009060480190012402F09EFB029061480078AA
S31900005424012101435F4801700098007A072801DA092500E0C6
S319000054380F2502F0EBFB0600742003F0BBFE854201D3002E3F
S3190000544C5ED10020009908720099C860009908610025019863
S3190000546000880121A94008421BD050480078C008204209D057
S31900005474F8680480083002F0F3FB54217854785C00287BD09A
S319000054882800FFF7C5FE002807D00098007A401C00990872A9
S3190000549C280003F0AFFE6D1CEDB20C2DD9DB0098C068400019
S319000054B0009948600098017A002909D000690A225043FFF76E
S319000054C44AF9401D0A21FFF746F900E00F200099088004F0AA
S319000054D885F8002809D002F03CFB3349096802F03BFB0628D0
S319000054ECF7D304F0D9F83048007801990979884201D104F07B
S31900005500C5F904F0B9FA01E0FFF7D8FD2A4801F042FF0028B4
S31900005514F8D129480078012811D10198007E04F0D5FA01984D
S31900005528007E001D01990876C0B2102805D1002001990876FE
S3190000553C02201F49087002F00AFB029902F00AFB0100F86869
S31900005550142909D30480083002F084FB54217854785C0028BE
S319000055640AD10BE01422511A0180083002F078FB5421785467
S31900005578785C002800D04CE702211037380002F079FBF7BD5E
S3190000558C24F2FF1FE4240020CDAB0000341B002084F00F40FF
S319000055A0B8040020A81A0020FC070020511F0020F007002069
S319000055B430F2FF1F981E00200608002010B50200002300208F
S319000055C803E0D45C001980B25B1CDBB28B42F8D310BD38B515
S319000055DC05000C00FFF7EEFF29190A786B465A706A46497811
S319000055F0117069460988814201D0002032BD012032BD38B540
S3190000560405000C00FFF7DAFF69460880281949780170694653
S319000056180978417031BD0000002901D0042901DB094870474D
S3190000562C902252008000084B181880180288074B134089000D
S319000056400C220A401A430280002004490870704704800000D9
S3190000565458FBFF1FF3FF000055FBFF1F80B50178052902D0BD
S31900005668072904D007E0401C00F008F802BD401C00F020FACC
S3190000567C02BD012002BD0000F0B585B0050068780390A87803
S3190000569004900398802805D0302801DBA948A7E0C7B200E04F
S319000056A40027A84990204000BA008A18101830227A43A54B61
S319000056B89A18009216462636FF22E632891801242A78022A0F
S319000056CC00D1B9E00A2A00D1E8E00B2A00D1D8E00C2A00D1C8
S319000056E09FE03A2A00D1E7E0432A00D104E14A2A00D17FE06E
S319000056F4512A00D1E4E0A22A00D1BCE0A62A05D0A92A00D10A
S31900005708AAE1AA2A00D0AC2A00D111E1AD2A00D1B7E0AE2AA8
S3190000571C00D1AAE0AF2A00D0B8E1E979032903DB4E2901D022
S3190000573087485DE0297A4E292AD00A07120F042A19DA028862
S3190000574413059B0F0C07240FA34212D0804B13408902C022F1
S3190000575812010A401A430280B17F202907DA009949314978CD
S3190000576C04220A43009949314A70297A0909052908DA028894
S31900005780754B13400903E022D2010A401A430280E9794E2919
S3190000579408D00288C04B13400902C02292000A401A43028093
S319000057A8E87801A94870287969460871022268468188380049
S319000057BC00F0FDFB69793800FFF72CFFA979380000F0AEFCBC
S319000057D00400A978380000F048FC20432CD17F1CFFB2302F23
S319000057E403DA0398802800D15BE7002005B0F0BDE87801A9EC
S319000057F84870287969460871002268468188380000F0D7FB43
S3190000580C69793800FFF706FFA978380000F027FC00280BD1FD
S31900005820DDE7E978380000F081FC0400A978380000F01BFC40
S319000058342043D2D0052203213800FEF72DFCCCE70188964A98
S319000058480A4004990C40A10111430180052203213800FEF724
S3190000585C1FFC009849300078FE21014000984930017000208C
S319000058708C490870B3E7032200E00122B07F2028B5DA307C5D
S31900005884032803D1B1E7022200E00022A87801A94870E8786B
S319000058986946087168468188380000F08AFB9AE70499C9B2D1
S319000058AC3800FFF7B7FE00289CD192E7002030757075B07522
S319000058C0B0748CE7009949310978049AD2070BD58A09224255
S319000058D483D101220A43009949310A7001880C4304807AE7AC
S319000058E8C1200142FBD0FE20084000994931BCE70398802858
S319000058FC01D16A4876E748780009204201D1FF20E870A8781D
S31900005910602802DBFF2806D102E0E978602904DBE978FF29E6
S3190000592401D0614862E77900604A51180870E878487052E751
S319000059380878810921420DD15C4855E70880000058FBFF1F31
S3190000594C30F2FF1F06800000FFF30000FF8F0000C00907D05B
S3190000596004988107890F3800FFF75AFE0028E8D12878A6289C
S3190000597401D1347001E002203070707B800719D10098493093
S3190000598800784007800F03D002280BD005D30FE0707B032109
S3190000599C014371730AE0707BFC210140012003E0707BFC218A
S319000059B00140022008437073717BF3200840AA78530601D5B4
S319000059C4910903E08907890F022901D0890000E00421014356
S319000059D871732878AC2801D1002003E0E879652800DB64203B
S319000059EC3073EA1C3900287800F0CEFB2878AC2821D1A878E0
S31900005A00042101406A465172082108406946087200200021D8
S31900005A14737BEF221A400901114371736946097A002901D0B1
S31900005A2800213170002801D0032030706846407A002801D085
S31900005A3C1E480470CDE62A7A012111406B46597202211140BC
S31900005A501972A628DCD15007C00F1107C90FD9E7009849304F
S31900005A64C078FE210140A878012202400A4300984930C2707B
S31900005A78B07F03280BD100984930C078FD210140E878044092
S31900005A8C6000084300994931C870A2E68020A9E6FFFC000058
S31900005AA0BFFF000055FBFF1F0A8000000980000098050020F0
S31900005AB40C80000002080020FEB505000024974897490191F5
S31900005AC89749984A0292F822072601272B78052B00D1C1E0BA
S31900005ADC092B00D118E10B2B00D1B6E02B2B00D182E03D2B24
S31900005AF000D1F6E0432B00D1F7E0552B00D1DFE0562B26D058
S31900005B04632B1BD0872B08D0A12B00D114E1BA2B00D121E13A
S31900005B18BB2B74D04CE16A780C2A01DBA648FEBDEB780A21F1
S31900005B2C5943008888424CD3A3485200B64B9A1811523CE1E2
S31900005B4068786A465070A878107068460088888033E1687829
S31900005B54162811D0282804D02E281AD032282AD02FE0A87831
S31900005B68052806DA0199097A0A4006401643019806721EE100
S31900005B7CA8780628FBDA01990979F0220A400007000F10430B
S31900005B900199087111E1A878002806D18A490F700198407933
S31900005BA4BF21014005E0FDF74BFD0198407940210143019815
S31900005BB84171A878002802D10120FFF737F86978C8080B28DC
S31900005BCC01D37F48FEBD0E40B740EF70F02149008D4A10186C
S31900005BE040180178AA78002A01D00F4390E0B9430170E2E0CC
S31900005BF401980078024068780640164301980670D9E0A978DC
S31900005C086A465170E97811706978042909DB08216970808A31
S31900005C1C6946098888420ED2694608800BE0408A128890422C
S31900005C3001D26A461080002903D168460088029988818320CD
S31900005C44400069784900724A51186A4612880A52B1E0681CFC
S31900005C5800F0BEF80400ACE06878FF281DD0AA78FF2A1AD0D3
S31900005C6C64230A260A2801DA6E7002E0652800DB6B700A2A23
S31900005C8001DAAE7002E0652A00DBAB70A8786A78824202D30F
S31900005C940A70A87801E00870687848708BE0E8780028FBD0AD
S31900005CA82A79002AF8D0904202D38A70E87801E088702879D2
S31900005CBCC8707CE0687800280BD1A878552808D1E878002858
S31900005CD005D12879552802D1002000F05DF9A94C6BE068786D
S31900005CE43A49087067E03A480078C008384201D0A44C60E027
S31900005CF8A44D280000F098F900280BD060222900A14801F070
S31900005D0CF3FCA148077052E06878C11E3A2909D3284C4CE05E
S31900005D20BE17000038FDFF1FBEFDFF1F5AFCFF1FFA21890050
S31900005D344143029801803EE068786A465070A87810706846FA
S31900005D480088C880E8785070287910706846008808812EE063
S31900005D5C687800281ED0572826D1E8786946487028790870E1
S31900005D70A878000127490818694609880A22514341816979C4
S31900005D840173A9794173E9796A465170297A11706946098884
S31900005D980A225143C1810CE0A87869464870E87808706846F6
S31900005DAC00889B49488002E03C0200E080242000FEBD00002A
S31900005DC0018000004E020000020800200380000001F2FF1F3A
S31900005DD4511F0020F0B585B000210D4B0278572A41D05F2A3D
S31900005DE803D0A72A00D1BAE0C5E04478072C03DB802C01D0A3
S31900005DFC4E2C3DD18278042A08DB802A06D04E2A04D0844862
S31900005E1029E000BF58FBFF1FC278052A03DB802A01D04E2A05
S31900005E244FD17F4A9A184E2C00D0147083784E2B12D05478D9
S31900005E389C420FD0537030234B43794CE31844331C78202CD8
S31900005E4C03DA9C79042525439D71491C3029F0DBC0784E2874
S31900005E6000D09070002005B0F0BD44782200103A702A03D33E
S31900005E74912C03DBFF2C26D06B48F2E782786D466A70C2780B
S31900005E882A7002AA2D88158005796E467570457935706D4643
S31900005E9C2D88558085797570C57935706D462D8895802501F9
S31900005EB05B190093007AFF280AD1D888D0801088974B984251
S31900005EC408DB9748CDE7FEF7ACFEC9E70A234343D380F2E720
S31900005ED80A23584310806500914840190190112C05DB10887B
S31900005EECFF21C943019A5052B6E79688A048A14B9E420FD1E4
S31900005F00009EB688968056889E4213D10098408850809088AB
S31900005F141E305288904210DB9948A2E75788B74201D217481A
S31900005F289DE74788BE42EAD2954898E70088B042EBD29448E1
S31900005F3C93E794480170082202A9009801F0D4FB0098008837
S31900005F500199088031480021415E2000FEF77EFEB3494853B4
S31900005F647EE74178090159180A7AFC23134080788007800F86
S31900005F781843087272E78020400070E704800000F0FF000037
S31900005F8C9805002042FDFF1F1905002080B5FDF783FAA54810
S31900005FA00068817801220A438270BFF34F8FA248A249086057
S31900005FB4BFF34F8FFEE730B50500080014006F49884227D0DF
S31900005FC8002C01D0012C01D1642100E01421FEF7BDFB30212B
S31900005FDC6943124A51184431002C05D0022C03D013D3032CAE
S31900005FF011D030BD91225200AB00914CE3189852087820288F
S3190000600403DA8879042202438A7100205F49087030BD488049
S3190000601830BD0000B8060020028000004A02000030F2FF1F95
S3190000602C0180000010B598B004006846602100F0FBFD302061
S3190000604002212278602A08DA6B469A181378002B01D0002013
S3190000605407E001231370641C491EF0D1401EEDD1012018B0F7
S3190000606810BDF1B581B04E2901D10020F6BD08090022002506
S3190000607C90235B006C462479A4006E4E3419E31801240F28A9
S3190000609001D0002819D11F886A4E3E4001270F4037431F80A6
S319000060A4274200D101256E46367930277E43654FBE190096E6
S319000060B849363778FE263E40009F49373E700F2801D0012800
S319000060CC0CD11E885E4F3740BC464E08760002273E406746F1
S319000060E03E431E800F2801D002280BD11E88584D35408E0823
S319000060F4F701802637402F431F8001250F2801D0032806D13C
S3190000610818884004400CC908C903014319801E4802702800D3
S3190000611CF6BD00007117000003800000E006002070B502007E
S319000061300023002003291EDA902464009500404E75192C19E0
S3190000614425882E06360FB607B60F8E4211D0404828400901EE
S3190000615830250D4005432580012030214A4338498918492212
S3190000616C8A5CFE24144049310C7006490B7070BDC4170000F5
S31900006180FFFF000007800000058000000680000055FBFF1F07
S3190000619470B582B00600140030204143294845180A2128008B
S319000061A8283000F041FD0020A62E04D0AA2E0DD0AC2E17D019
S319000061BC73BD207869464870684661780170008828856846BF
S319000061D0008809E0215C8A0051184200AA181185401C0428B2
S319000061E4F6DB288DA88673BD6946225C0A70A1796A4651708B
S319000061F8042801D1617951704210920F121892109200811A08
S3190000620C4906090E6A46527803238B401340CB4069464B70DF
S3190000622009884200AA181185401C0528DEDB73BDC0060020E1
S3190000623424F2FF1F0400FA050CED00E058FBFF1FFEFF0000D2
S3190000624830F2FF1FFDFF00007FFF0000CFFF000008B4024BAB
S3190000625C9C4608BC6047C0464DF1FF1FF8B500210024022560
S31900006270324F01260278062A1AD0072A49D02D2A2CD0412AD0
S319000062843FD0FF2A56D100BF38A243185B78555CAB4202D06A
S31900006298F0030843F2BD491CC9B20529F3D3002000F056F8CD
S319000062AC2000F2BD40780F283ED122480078C008304212D10C
S319000062C020480178491C017003F064FC0028EDD178780421BF
S319000062D4014379700124E7E718480078C008304201D0184C49
S319000062E8E0E703F091FD03F051FC002802D015480570D7E78A
S319000062FC7878082101437970D2E74078114A1070114801702C
S31900006310CCE7407801280DD1FEF71DFCFA218900884203DAA8
S319000063240120FEF7B1FABFE7787805437D70BBE78024B9E7ED
S319000063380120F2BDE4240020511F002000080020F0FF0000AC
S3190000634C1905002058FCFF1F55FBFF1F10B50400FFF701F861
S319000063602000FDF79FF8FFF777FF00F04AFAFEE79915161619
S319000063749900000080B50178042902D0072904D007E0401C82
S3190000638800F007F802BD401C00F024F802BD012002BD1CB575
S3190000639C00240178532918D120490988012243799A401142DF
S319000063B012D0C1786A465170694602790A7001A96A461288AF
S319000063C44A8042790A70807848700320FEF79AFD00E08024DD
S319000063D8200016BD010000200A78C22A1DD14A781202897864
S319000063EC0A430F498A4217D101210E4A127852080A4203D1C0
S319000064000B210C4A117070470B4A53780B4209D11943517064
S3190000641403211170517802230B4353707047802070470000BC
S31900006428341B00209B90000039FDFF1F54FBFF1F19050020C1
S3190000643C08B4024B9C4608BC6047C0464DF1FF1F08B4024B85
S319000064509C4608BC6047C0465DF1FF1F10B5A84C1821200061
S3190000646400F0E6FB00F0F4FB0F2000F05CFD80093C210140CF
S31900006478A181084604D00121A17203F099FD04E0A07296205C
S3190000648CC00103F009FE60229B499C48FEF780FB10BD80B57F
S319000064A0FFF7CCFF002000F0E3FB002000F031FC93480021FA
S319000064B401728089C0B203F07DFDFFF7C5FF01BDF8B5060048
S319000064C80F0014000125002C04D18E4841780D434570F1BD2E
S319000064DC8848807A012801D1FFF7AAFF3900300000F0D2FB1C
S319000064F001280ED1002E03D18148807A002801D0012E02D1CA
S31900006504300003F051FE3900300000F0C6FB7F1C641EA4B27E
S31900006518002CE5D17848807A012801D1FFF792FF002E0ED13E
S3190000652C7448807A00280DD001280DD1994800788009284247
S3190000654008D0082097490860F1BD012E02D1012003F02CFE0B
S31900006554F1BD70B5040000F0E2FB0F2803DB200000F07AF8F2
S3190000656870BD00281CD06448A10046180519287A002805D16F
S3190000657C01F0EDFA30600120287270BDFA214900306801F0C8
S31900006590F0FA002808D0FFF751FF00202872200000F0B7FB45
S319000065A4FFF752FF70BDF1B582B0012708240025524E7A48B6
S319000065B80078C00838421DD0307D002804D03575377601F031
S319000065CCC6FA3061307E002812D074480188306901F0C9FA1A
S319000065E000280BD071480068817808220A438270FFF755FFD1
S319000065F46E4804603576F7BD6846007A00F08FFB0F2804DB5C
S319000066086846007A00F026F8F7BD002821D06846007A8100CC
S3190000661C711800913618307A012805D001F097FA00990860D1
S319000066303772F7BDFA2149000098006801F099FA00280AD009
S31900006644FFF7FAFE3572594804606846007A00F05EFBFFF73B
S31900006658F9FEF7BDF0B585B0040000260025264F01207875D1
S3190000666C6946200000F072FB6846007801A948556D1C0F2DB6
S31900006680F4DB210001A8FCF7CBFA787D002807D00F256946D8
S31900006694200000F057FB6D1E03D0F8E7200000F0EAFA381908
S319000066A8067205B0F0BD012013490875704780B53E4902206F
S319000066BC03224B781340012B06D13C4B1B789B070ED40B21BC
S319000066D03A4A11703A490A78104308700848807A012808D18F
S319000066E40020FFF760FF01BD0A704A781043487001BD002044
S319000066F8FFF72DFF01BD0000AC07002042FDFF1F98050020BB
S3190000670CE424002070B52C4DE868083001F0A4FA5421685465
S31900006720685C0028284C0AD170BD01210180083001F098FA99
S3190000673454216854685C002829D001F00CFA0600FFF7B7FF8C
S3190000674803F04CFD03F08AFFA07D401CA075C0B20921FDF761
S3190000675CFBFF002903D100F00CFA0020A07501F0F6F93100F0
S3190000677001F0F6F90100E8680729D6D20722511A01800830B9
S3190000678401F06EFA54216854685C0028D5D10221103528004F
S3190000679801F070FA00BF00003BFDFF1F88F00F405AFCFF1F3C
S319000067AC24F2FF1F84F00F401905002039FDFF1F54FBFF1FDD
S319000067C0FC070020B8040020AC07002080B597484178491CBB
S319000067D4C9B20B2906D102781207120F0F2A01D100210170D4
S319000067E8417040780B2801DA00F026FA01BD00208C4A50709C
S319000067FC8C490860704780B58B488A49086000F019FABFF397
S319000068104F8F894889490860BFF34F8FFEE7884800680028B0
S3190000682400D1704780B5C06A007885490978884201D000F021
S3190000683801F801BDB0B588B0002502A834A11022FEF7BCF972
S3190000684C01A800BF35A10A680260002402A8032141717849BB
S319000068600968C96A0978817176490978C1710021425CAD1811
S31900006874ADB2491C0D29F9D3290A4173857301AF00F0DCF9F0
S319000068880F2202A90020FFF719FE01F062F905006B48807AEF
S3190000689C002816D0002000F0F2F90028FAD1694600F04CFA01
S319000068B00028F5D168460078395D884201D00024EEE7641C10
S319000068C4E4B2042CEADB19E00024FA218900280001F04DF90F
S319000068D80028D3D100F0D5F90028F4D1694600F02FFA00283F
S319000068ECEFD168460078395D8842E9D1641CE4B2042CE6DB8B
S31900006900FFF79CFDAD480068C17801220A43C270FFF777FF4A
S3190000691408B0B0BD03FF024E4E4E4E4E4E4E4E4E4E00000034
S31900006928454E5452F3B58DB03022FF2101A8FEF727F93022B5
S3190000693CFF210D98FEF722F90020002130224A439C4B9A18B3
S319000069504A3212789207920F01AB5A540D9B5954491C302980
S31900006964F0DB411C0D9A121801AB1B18009333E0009B1C786C
S3190000697801AB5D182E780D9B5B18A64206D2009F3E702C707A
S3190000698C14781E7816701C70009C24782D78AC421DD1147878
S319000069A01D78A54201D215701C700EAC2478002C13D014788C
S319000069B430256543814E751936352D78102D0ADB1D78302652
S319000069C86E437D4FBE1936363678102E01DA15701C70491CB8
S319000069DC3029C9DB401C2F28BFDB0FB0F0BD30B50020754928
S319000069F030224243724B9A184A23D45CFC2323409024640010
S31900006A0485004D192C5B2406A40EA407A40F1C434A3214706D
S31900006A18401C3028E8DB30BD67490A8A104308827047000028
S31900006A2CFC07002000F0FF1F5A876A950400FA050CED00E063
S31900006A4028F2FF1FBC170000AC070020F3B581B011001E0056
S31900006A54002468460079FCF763FA07000125002E6AD068464A
S31900006A68017A0079FCF75AFA0600052F01DB2B2F0CD1062E58
S31900006A7C02DB2B2E04D107E0032E05D1042F03D10120FFF7E9
S31900006A90C7FF0124B74220D01C2F09D01F2F05D0252F05D0A8
S31900006AA4312F01D04A2F16D1202011E045480078800928421E
S31900006AB80BD068460079302148433F4908184A300078C00686
S31900006ACC800F032803D00420FFF7A4FF0124052E01DB2B2ED9
S31900006AE03DD1062F07DB2B2F05D0452F03D00220FFF796FF54
S31900006AF401241E3F1CD07F1E18D07F1E1AD0113F14D07F1E3D
S31900006B0816D0BF1E012F0FD93F1F012F0CD93F1F032F0DD9AF
S31900006B1C083F012F06D93F1F06D07F1E06D07F1E012F16D8A7
S31900006B30082011E010200FE040200DE01F3F012F09D9FF1F38
S31900006B4407D00B3F012F04D90B3F032F01D9FF1F03D1802021
S31900006B58FFF762FF01E0002C0CD068460079C0081549081876
S31900006B6C817C6A4612795207520F95400D438574F7BD1048F3
S31900006B80008A12490988084204D01148016810220A430260C4
S31900006B94704780B5FFF750FC08480021018206221230FDF767
S31900006BA8EFFFFFF74FFC0848016810229143016001BD0000C6
S31900006BBC24F2FF1F30F2FF1F58FBFF1F40FDFF1FC2FDFF1FA2
S31900006BD094F00F401206130A1A43130C1A4300BF094205D0EB
S31900006BE483070BD00270401C491EF9D1704700001206130A47
S31900006BF81A43130C1A4300BF130030B414001500103902D3AD
S31900006C0C10393CC0FCD2490700D30CC000D504C0890002D375
S31900006C200280801C002900D5027030BC704700000022D5E74B
S31900006C340022E3E70C20044908607047034855210160AA21D5
S31900006C4801607047008104400481044080B5002000F00AF845
S31900006C5C002000F058F8012000F004F8012000F052F801BD98
S31900006C7080B5142148433D494FE080B51421484339490818C9
S31900006C8400F0DEFB01BD80B51421484336494AE080B5142266
S31900006C985043344A4DE080B514225043314A101800F077FBA1
S31900006CAC01BD70B5040016002D48002C1BD1002919D02C4CBA
S31900006CC021780025002901D0481E05E0310000F090FB0028E3
S31900006CD403D10E202070357007E00020FFF7D3FF002802D1A5
S31900006CE8082022490860002070BD310014226243801800F0B6
S31900006CFC7AFB002802D10020C04370BD2000FFF7BEFF00B239
S31900006D1070BD80B5142148431349081800F02DFB01BD80B5C0
S31900006D24142148430F49081800F033FB02BD80B51422504342
S31900006D380B4A101800F02DFB401E8041C00F02BD80B5142294
S31900006D4C5043064A101800F04EFBF3E780B514225043024AC5
S31900006D60101800F07AFBEBE79CF1FF1F74F1FF1F0408002060
S31900006D7484F00F4038B500240025200000F008F82D18ADB258
S31900006D88641C302CF7DB3448C58031BD38B5040030216143AE
S31900006D9C304A55183635A97B202902DB2978032912D1FDF79D
S31900006DB091F8002803D0022805D002D30AE0288B32BD288A33
S31900006DC432BD91204000A100254A5118085A32BD002032BDFC
S31900006DD838B5FFF7CDFF20482149027852008A5AC388204CB9
S31900006DEC00259A4203D2002225786D1C00E0D21A257002818B
S31900006E002278042A06DB00784000085A181A80B200F001F868
S31900006E1431BD70B58CB000250A3086B201216846FFF782FD39
S31900006E28302468460019401E0078302141430A4A5118443158
S31900006E3C0A78202A08DA49886D18ADB208220321FDF726F978
S31900006E50B54203D2641EE4B2002CE6D10CB070BD30F2FF1F38
S31900006E6458FBFF1FC006002005080020704718B402E0401CCF
S31900006E78491C521E002A09D00B7804789C42F6D002D2002091
S31900006E8CC04302E0012000E0002012BC7047000080B52C48B8
S31900006EA00168802212050A4302602A480021016064228260AB
S31900006EB4C160012101620721416200F001F801BDF0B523489C
S31900006EC88021426A0A43426202680A40FCD0416A490620D404
S31900006EDCC76C866C426C036CC46B856B80210902BE19B218EE
S31900006EF0D218121952191204520C0A43C262C76E866E426E4A
S31900006F04036EC46D856DBE19B218D218121952191204520C4A
S31900006F1811430163F0BD0E48017810220A430270F0BD1F2846
S31900006F2C01DB0020704708490A681F239A430A600A68104387
S31900006F40086008680006FCD5086980B2704700003C8004402E
S31900006F5400B00340E424002080B56F4AA821102001F028FF09
S31900006F680A2000F058FE00210C2000F093FA01BDF3B585B03A
S31900006F7C002001900427C02260216648FFF734FE6846007DBB
S31900006F90002801D1FFF7E2FF02229C21102001F00BFF0025E5
S31900006FA400246B4601229C21200001F017FF68460088022897
S31900006FB800D07EE06B4601229D21200001F00CFF0120A040E2
S31900006FCC694608816846008800280FD06846008838420698E8
S31900006FE005D08088098901430698818004E0408809890143C3
S31900006FF40698418003AB01229E21200001F0EEFE06206043CE
S31900007008C2490E1868468089400A0321B278FC231340032257
S3190000701C02401A43B2706A46928932800C2201408800101AFB
S319000070306946887068468078042813D102203071B178C3201A
S319000070440840694689788A003C2111400143B1708806800E81
S31900007058090989010143B170002047E008281BD16B460122E6
S3190000706CD721200001F0B6FE68460088C00501D5002002E07A
S319000070806846877001203071F07869460988890503D501215F
S319000070940143F170D2E7FE210140FAE70121A140C843069996
S319000070A889880140069A918006994988084006994880641C2C
S319000070BCE4B20C2C00DA70E706980088002806D00198401CA2
S319000070D0C0B20190022800D053E707B0F0BD22010107090FC8
S319000070E411438C4AEDB28A4B5B1999546D1C401CB1788906F6
S319000070F8090FC0B28842EED306980088694609890143069820
S3190000710C018001980028D2D11E2000F082FDD3E7CDAB0000A5
S31900007120BC1A0020F1B584B06846007C0C2805D10026039098
S3190000713410206946087404E06846067C701CC0B2039000221F
S31900007148AA216846007C01F033FE1822C8216846007C01F0D8
S3190000715C2DFE6F4AC9216846007C01F027FE6D4ACA216846BB
S31900007170007C01F021FE6B4AA9216846007C01F01BFE694C11
S319000071842200F6216846007C01F014FE2200F7216846007C27
S3190000719801F00EFEFF242401220008216846007C01F006FE2E
S319000071AC22003A216846007C01F000FE64E05C4800880121A1
S319000071C0B14008425DD06C2070435249081802906846007C97
S319000071D4102829D1002400256B46012229002E39C9B2F0B2A5
S319000071E801F0FAFD0020694609888200D1400907090F6A46DA
S319000071FC5180E4B24FA31B5D591A06237343424FFB5A484FD9
S31900007210BB4200D10021029B1A1956321170401C641C042894
S31900007224E3DB6D1C022DD7DB6B460122D721F0B201F0D4FDF8
S31900007238684600880299A03108706B4604221221F0B201F085
S3190000724CC9FD6B4604224421F0B201F0C3FD6B460122982146
S31900007260F0B201F0BDFD68460088324901400C2008436946AF
S319000072740880684602889821F0B201F09BFD761C0398864267
S3190000728897DB2B4A99216846007C01F091FD80221202972134
S3190000729C6846007C01F08AFD002201216846007C01F084FD56
S319000072B0002233216846007C01F07EFD002265216846007CE6
S319000072C401F078FD00242200A6216846007C01F071FD641C34
S319000072D8042CF6DB02229C216846007C01F068FD002406E030
S319000072EC42886846007C01F061FD641CE4B2D5208000A10019
S319000073000E4A511808180178FF2901D0102CEDDB05B0F0BDBA
S31900007314501500206C0500003759000082BF0000FFFF00009A
S3190000732849020000341B0020C24A0000C0FF00002C0A000090
S3190000733C281500000B08090707070809F8B504000F001500E3
S319000073501E00FFF773F82660277128007843E0800020208182
S319000073647D43E91B61816189E181207360732082FFF76AF8BD
S31900007378F1BD10B50400FFF75DF800202081E1882279891AD1
S3190000738C6181E181207360735DE0407B704738B504000D0090
S319000073A0FFF74CF8207B002803D0FFF74FF8002032BD22791C
S319000073B4290020892368181800F09AF9208921794018208173
S319000073C880B2E188FDF7C2F92181607B401C6073208A401CAF
S319000073DC208220896189884201D101202073FFF72FF80120D4
S319000073F032BDF8B504000E000025FFF71FF8607B00281BD0B5
S3190000740427796089C019608180B2E188FDF7A0F961813A00E7
S31900007418608921680918300000F068F9607B401E6073C0B2C8
S3190000742C218A884202D220826089E08125730125FFF706F85F
S319000074402800F2BD10B50400FEF7F8FF6089E081607B2082DF
S31900007454FEF7FAFF10BD70B504000D000026FEF7EBFF208A7E
S31900007468002813D02679E0898019E08180B2E188FDF76CF909
S3190000747CE1813200E08921680918280000F034F9208A401E02
S3190000749020820126FEF7DAFF300070BD80B50A009A211020C4
S319000074A401F088FC01BD80B542884178007801F081FC01BD3F
S319000074B880B5831C01224178007801F08DFC01BDF2B582B081
S319000074CC0500802809D100246846017A200000F04DF8641CFD
S319000074E00C2C45DAF6E7290081390D2907D26846017A28001B
S319000074F47F30C0B200F03EF838E05549554A101840180090D2
S319000075080078040953490A88E240D20703D44988E140C90722
S3190000751C28D501270F2601223040824092B2A521200001F08B
S3190000753043FC280000F083F80098027810460F2111408900FD
S3190000754412096C235A43434B9A18511880310640B20000098B
S319000075586C2358433E4B18188018803000686A46127A974073
S3190000756C07430F602800FDF707FFF7BDDAB582B00400374832
S3190000758000880121A140084258D0354E3200A521200001F068
S3190000759411FC334F3A00F621200001F00BFC3A00F721200073
S319000075A801F006FC6B4601220821200001F014FC6846008882
S319000075BC304069460880684602880821200001F0F5FB6B46FB
S319000075D001223A21200001F003FC6846008806406846068063
S319000075E432463A21200001F0E5FB6B4604221221200001F0AE
S319000075F8F3FB6B4604224421200001F0EDFB00200FE08100C6
S3190000760C6C226243114B9A18511880310A686B461B7A01262A
S319000076209E4016430E60401CC0B2062161430A4A5118897854
S319000076348906090F8842E6DBDFBD80B50449054A1018405CD9
S319000076480107090F000900F00BF801BD6C0500005015002058
S3190000765C341B0020FF0F000049020000F8B507000D00AC08D7
S31900007670694620000A3888706B46012268468178380001F053
S31900007684ADFBAE07B60F700080190125694609880722824070
S319000076989143012282400A436846028002888178380001F0F6
S319000076AC85FB684632216143083181706B4601228178380070
S319000076C001F08EFB6846018830000C308540A94368460180B3
S319000076D402888178380001F06DFB6B46012232204443A11921
S319000076E81231C9B2380001F077FBF1BD10B50400FDF750FA7A
S319000076FC200010BDFFB585B0012669464E726846077EAD48E0
S31900007710AD497B00DB19C318591803916946097D0491AA4B5B
S31900007724591801916946097F002903D0022925D00ED330E004
S31900007738002501240398027868464572019801796846037E31
S3190000774C01209840814320E002249E490978314205D0022569
S3190000776003249C49C019425C0EE09B49405C304202D00225B3
S31900007774032400E001250398427803E00325042403988278B1
S319000077880198007969460B7E012199400143019801715620DD
S3190000779C04996C2359438E4B5918C91908567A21091A7A2029
S319000077B0424348101018FCF7D0FF0190FF2801D9FF200190B6
S319000077C46846007E80086946C8706846C0783221484369469D
S319000077D80872B907890F49084718BF1D6B460122F9B268460C
S319000077EC007D01F0F7FA6846007E01210140C800694609888D
S31900007800FF2282409143019AD2B282400A43684602800288CF
S31900007814F9B2007D01F0CEFA6B4601226846017A007D01F00E
S31900007828DBFA6846007E8007800F69468870684680784000A2
S3190000783C0988032282409143EDB285400D4368460580028875
S31900007850017A007D01F0B0FA08A8007800281BD06846C77863
S319000078640A3F6B460122F9B2007D01F0B7FA6846807841003C
S31900007878081869460988072282409143E4B284400C43684680
S3190000788C04800288F9B2007D01F090FA6846C478322044436E
S319000078A008346B460122E1B26846007D01F098FA68468078D7
S319000078B486406846407A00286846008803D0064368460680DE
S319000078C802E0B0436946088068460288E1B2007D01F06EFAF9
S319000078DC09B0F0BDF8B507000D001400AE08322046436B4615
S319000078F00122F1B2380001F073FAA807800F0830694609886C
S3190000790401228240914384400C43684604800288F1B2380006
S3190000791801F04EFAF1BDF8B52A4C2078401C207000252582FB
S3190000792CC0B20A21FCF710FF002925D100207E49002203E097
S31900007940BE1B1E70521CD2B206234343234EF3189B789B06F5
S319000079541B0F9A4211DA231D1B5C01269640334201D04E7868
S3190000796800E00E78C300724FFB189B181F78B742E2D21D7084
S3190000797CE2E7401C0C28DBDB00216D4800F025F9052000F0E9
S319000079901FF900F02BF9F1BD0C4A1218127901238B401A42AD
S319000079A404D1C000634A101800224254704780B5002005494D
S319000079B8087060215E48FFF739F901BD281500001E030000D2
S319000079CCC80700203EFDFF1F360300004E030000501500204A
S319000079E0E0B588B05648008A242802DA00F0FEF805E000F0B5
S319000079F403F900211120FDF7E8FA00274C4801904F480088EA
S31900007A080121B940084200D185E00026F6430025F8004749BD
S31900007A1C081800906C20784348490818049006207843081813
S31900007A30039004E00078101808706D1CEDB203988178880663
S31900007A44000F85422DDA6810800F401980108000281A029007
S31900007A580DD1761C880936B28642EADA05AB012232217143C5
S31900007A6C1731C9B2F8B201F0B5F90123AB4004984A30008847
S31900007A801842DAD06846828A0299012088400242D3D000982B
S31900007A9441190A782C48C05D18420198C8D04078C7E7002159
S31900007AA8002200250CE0009B5B5DC918C9B2002B04D01300D0
S31900007ABC0122AA401A4392B26D1CEDB28542F0DB01984088E7
S31900007AD0884224D2A521F8B201F06EF93820184908820025AC
S31900007AE415E000984019017800290ED0002101702900F8B2BD
S31900007AF8FFF7B6FDA8000499081880300168802252030A4309
S31900007B0C02606D1CEDB2039880788006000F8542E3DB7F1C8D
S31900007B200C2F00DA6EE70648008A401C0449088208B0E0BD81
S31900007B34BE180000F8050020E1790000C8070020341B00208C
S31900007B4850150020CC07002041480168491C016070473F48B5
S31900007B5C00687047884201D3401A70470022D243511A08187F
S31900007B70704710B50C00010037480068FFF7F0FF844201D20D
S31900007B84012010BD002010BD38B5334CE068083000F066F8D2
S31900007B9854216054605C00282D4D04D131BD6868010000D0E8
S31900007BAC8047E06829890180083000F055F854216054605C23
S31900007BC00028F0D102211034200000F057F800BF214908814A
S31900007BD47047204A5060907AFD23034048000221084018434B
S31900007BE89072704780B51A48817A01220A438272018907E063
S31900007BFC80B51648817AFE220A40827215490181742001F01E
S31900007C104CF901BD1048817A8807C00F704738B504000D48A9
S31900007C24056821002800FFF7A2FF0028F9D031BD70B50400F1
S31900007C380D00002C09D00648066800E0A84721003000FFF74E
S31900007C4C92FF0028F8D070BD0000000010F2FF1FB804002074
S31900007C60FFFF0000F0C042464B4654465D466E467746FCC0D9
S31900007C742838F0C800207047002900D1491C1030FCC8BE46A0
S31900007C88B546AB46A246994690462838F0C808007047000082
S31900007C9CF0B583B0002690490E70182200218F48FCF76CFFE9
S31900007CB00022A121102001F07FF80022A221102001F07AF8C6
S31900007CC49022920000218848FCF75CFF002287488749411809
S31900007CD80191012581494978012911462CD1844B5B5C012B1F
S31900007CEC22D1834B4418E35C1C09019F3F88E7402F421BD013
S31900007D001A07120F6B461A706200764B9A1893889C460127F2
S31900007D146B461B789F4063461F43978001226B461B786C2716
S31900007D287C430419E318A1331E7001E0724C6654491C6029C1
S31900007D3C29DAD2E76D4B5B5C022B21D16C4B4418E35C1C096C
S31900007D50019F3F88E7402F4218D01A07120F6B461A70620053
S31900007D645F4B9A1893889C4601276B461B789F4063461F4356
S31900007D78978001226B461B786C277C430419E318A1331E70A7
S31900007D8C491C6029D6DB002A08D1FFF731FF524845700021A5
S31900007DA00020FDF714F9F7BD0024019800880121A140084262
S31900007DB407D060004A4908188288A121E0B200F0F9FF641C05
S31900007DC80C2CEEDB01214D48FFF701FF0120FFF7FBFEFFF7ED
S31900007DDC07FFF7BDF1B58AB000200090474E48480088012174
S31900007DF0009A914008426DD01046302148433B490818019020
S31900007E041022014620311030FCF7C6FE002500986C214843CE
S31900007E1835490818049050E005AB0822322169430E31C9B25B
S31900007E2C0098C0B200F0D6FFA80003900AA80078002819D1F6
S31900007E40002403980719600005A9085A8004400A04994831F5
S31900007E540A8831001140FCF77EFC711C884200D330003F06F4
S31900007E68F90D019A5052641C042CE6DB00240398071960000D
S31900007E7C05A9081802900089310001404802049948310A889F
S31900007E9031001140FCF761FC711C884200D33000FFB2790082
S31900007EA4019A511808840298028939000098C0B201F036FBAA
S31900007EB8641C042CDBDB6D1CEDB20098062148430949081866
S31900007ECC807880098542A5DB0098401C00900C2885DB0BB001
S31900007EE0F0BD0000E4F1FF1FE8F1FF1FC8FDFF1F5015002089
S31900007EF4E40500002C0200206C0500008C020020FD810000A0
S31900007F08FF030000341B0020F1B584B0A34BA44C6418E318BF
S31900007F1C0293B34B5B18FF20B63054246D462D7C002D03D06C
S31900007F30022D5FD02FD383E0252069468881DA2676003621AA
S31900007F440522029800780409019430256C43A74D2D19000703
S31900007F58000F6C4620706846007840002818048CA325AD0013
S31900007F6CAC4202D2058AAC420DD204201870019840009D4C6F
S31900007F802018858801246F463F78BC40A543858056E0601B77
S31900007F9452E069468C810600FD211B220298007804090194D0
S31900007FA830256C43904D2D190007000F6C462070684600781A
S31900007FBC40002818048C058AAC4202D20420187038E08A4DAF
S31900007FD0AC4201D305251D70058A641B6D466C80008CFF24C2
S31900007FE48834A0428041C043C00F6C46A07325E069468C81CC
S31900007FF806005A210922029800780409019430256C43794D45
S3190000800C2D190007000F6C4620706846007840002818048C86
S31900008020058AA54205D300256F467D70008A001B04E0012582
S319000080346F467D70008A201A6C4660801C78042C27D00298E5
S3190000804800780509019530277D43674F7D190007000F6F46D4
S3190000805C38706846007840002D5A684647888089684336040A
S31900008070360B80197843029069431204900B08180002062228
S31900008084082102266F463F7C002F03D0022F42D010D382E097
S3190000809802998842FBD20198400054490818818801226C4628
S319000080AC2478A24091438180012071E0029FB84210D2052C47
S319000080C000D01E706A4652882E246543DA2464012C19544385
S319000080D4844262D2187805283AD03DE0052C5CD069464988D7
S319000080E87B4C6C437B4EA4194C43844201D2032050E0694658
S319000080FC498891246543DB2464012C194C43844241D368467C
S31900008110807B00283DD0092040E0022C3FD0052C3DD0032C32
S319000081243BD06F467F78002F01D0092C2FD0029FB84216D2D3
S319000081381A781E706C4664882E267543DA267601AD1965437E
S3190000814C854207D2082A01D1197022E0072A20D107201DE0A4
S31900008160082A1CD101E0082C01D1052016E0072C01D11E7051
S3190000817413E06946498891267543DB267601AD194D4385427A
S3190000818805D2092C01D0062C05D11A7003E0062C01D1042063
S3190000819C187005B0F0BD00006C0500005015002070B50600BE
S319000081B000244B4D4B482919085C010901224A4BEB5ACB40AE
S319000081C413420CD04900484B591889880007000FC1401142A8
S319000081D803D0E1B23000FFF797FE641C602CE5DB70BD000073
S319000081EC8C020020C8FDFF1FE4F1FF1FD203000070B53B4E72
S319000082003B4831783B4A5118085CFFF7E1FCFFF7EDFC01250E
S319000082143078082857D801A1095C8F44080C1418484C5662E3
S319000082287000012225E00120FFF7D6FD4BE002221FE000204C
S3190000823CFFF7D0FD0020FFF7B3FF00242B4800880121A1407B
S31900008250084206D0600030188288A121200000F0ABFD641C48
S319000082640C2C32DAEEE7042205E00120FFF7B6FD012009E008
S319000082780822A221102000F09BFD24E00120FFF7ABFD022062
S3190000828CFFF78EFF1DE00022A221102000F08EFDFFF7AEFC28
S319000082A0707801280BD1401C707001211348FFF792FC012079
S319000082B4FFF78CFCFFF798FC07E0757000210020FCF783FE27
S319000082C801E0FFF797FC3078401C307070BD00003406000027
S319000082DCD01D0000501500206C050000E4050000E4F1FF1FC9
S319000082F09A03000028150000341B00209D7C000038B56A4C6F
S319000083040020207101252570657000F029F8002807D1FFF717
S3190000831871FCA57100210120FCF755FE31BD01216148FFF791
S3190000832C54FCA079012811D15F4A182120000830FEF75AFC3E
S3190000834022899F21102000F037FD0122A021102000F032FD31
S319000083540A2000E00120FFF739FCFFF745FC31BDFCB551484A
S31900008368FF218170C17052490091098800248279012A2FD1B2
S3190000837C0022002300254E4E4E4FFF18BE5D36090F00F7408D
S31900008390FE071DD5009E3669F6180196BD4EF718019E367893
S319000083A4F61E032E11D2D2B2022A0BDA8618B370521C019E34
S319000083B836787600761FF6B2B54205D2350003E087263E7009
S319000083CC00E03C705B1C602BD5DB4571120628E0012200233D
S319000083E0364D374EF618755D2D090E00EE40F50717D5009DA4
S319000083F42D69ED182E78B61F032E10D2D2B2022A0ADA861814
S31900008408B370521C2D786E000B3EF6B2B44204D2340002E0E3
S3190000841C87259D4EF5545B1C602BDBDB4471D2B2012A01D178
S319000084300020F6BD0120F6BDF8B514001A0006235C43E4B252
S319000084444300194DEB181D893F26A640B5431A4EB34F79188E
S31900008458895D0907090FA1402943241DA2400A431A8192B260
S3190000846C9F2100F0A3FCF1BD38B5114AAA4B5918895C0C0753
S31900008480240F002109198D086B460122322169431631C9B242
S3190000849400F0A4FC68460088A900611A4A005118C8404007E2
S319000084A8400F32BDC4F1FF1FC5840000FF0F0000341B0020E3
S319000084BC6C05000050150020F0B585B0974F38799EA1085C9C
S319000084D0FFF77EFBFFF78AFB00249448029038198678FF2E9A
S319000084E44ED092488E498919081803900078000969460870B2
S319000084F80298006880196549891901913D193979052975D86A
S3190000850C01A2525C974400BFC2067282B2C6310068460078DF
S31900008520FFF7A8FF042805D002990979002903D0042801DA83
S31900008534002100E00121297000011730019908700298006815
S31900008548805D032804D0062802D02878002848D0012203989F
S3190000855C00780007000F824092B2A5216846007800F024FC75
S319000085700323E2B2310068460078FFF75DFF3000FFF75DF813
S3190000858438E00178042921D005291FD007291BD11CE0007881
S31900008598042805D0052803D0072801D0082827D128780028D8
S319000085AC24D1310068460078FFF75EFF01990978C01F0818FC
S319000085C00199087011E00178052901D0082913D12878002849
S319000085D410D1012308E00078052801D0082809D12878002858
S319000085E806D10223E2B2310068460078FFF720FF641C022CCF
S319000085FC00DA6EE73879062816D1FFF7F9FAB87901280BD151
S31900008610401CB87101214748FFF7DDFA0120FFF7D7FAFFF76F
S31900008624E3FA32E00120B8710021FCF7CEFC2CE00122A02135
S31900008638102000F0BDFB002438198078FF2817D03949364AD3
S3190000864C1018405C0107090F019100225218950800AB9B1C13
S319000086602E0032225643AA00891A711812310122C9B2000925
S3190000867400F0B4FB641C022CE0DB38797979884201D106207F
S3190000868800E0401C387105B0F0BD00008C02002080B5274A3D
S3190000869C9F21102000F08AFB0122A021102000F085FB0021BA
S319000086B00620FCF78CFC01BD70B582B00400FEF703FF18489F
S319000086C41A490219561831780D091B49405AE840C00723D50C
S319000086D86B4601229F21280000F07EFB30780F210F22024018
S319000086EC6B461B881940914202D1FC21890001E090011049B0
S3190000870001436846018002889F21280000F054FB0122A02157
S31900008714280000F04FFB00200949085573BD00005015002065
S31900008728C4F1FF1F441B00206C05000001830000CF0300001E
S3190000873CE40500000F0C00008C0200200F090F090F09010028
S3190000875070B50600864D6E6200208649087086480178FE2273
S319000087640A40027001243079204214D082493278FF2A08D0B5
S319000087780A680023DB439A4201D012020A6032780A70B278BB
S3190000878CFF2A04D00A6812020A60B07808700022A121102032
S319000087A000F00AFB0022A221102000F005FB24212800FEF763
S319000087B43FFA300000F019F8287C204204D100210220FCF730
S319000087C802FC70BD686A01798907890F0C220A4302710121E8
S319000087DCBF48FFF7FAF90120FFF7F4F9FFF700FA70BDF1B5CC
S319000087F084B00020029002984000049908180190007802994E
S3190000880412225143594A5418FF2804D1207CFE2101402174F6
S31900008818A1E06070B04801990978B04A5118085C06090707FE
S3190000882C3F0F2670A770019840788007800FE0700020C01987
S3190000884081088800381A6A4690700D0032204543684680787E
S319000088542818123020713220414308001730607123000833A3
S3190000886801220D31C9B2300000F0B6FA208940026C2272431C
S3190000887C99498918483109888905890DFBF767FF8021C9006F
S31900008890884200D3481E20816B460122E9B2300000F09EFA03
S319000088A46846807840006946098803228240914300228240F5
S319000088B80A43684602800288E9B2300000F078FAA571012536
S319000088CC01984078810801200840227CFB2111408000084379
S319000088E02074019949780A0901211140E72202400801104362
S319000088F4012101432174002261787A4842546B460122A12186
S31900008908300000F069FA68460088BD400543AAB2A121300009
S3190000891C00F04CFA6B4601222179300000F05AFA6B46012255
S319000089309721300000F054FA68460088FF2109020140042041
S31900008944084369460880684602889721300000F031FA01213A
S319000089583000FEF79FFD0298401C0290022800DA45E705B0D7
S3190000896CF0BD00003007002003080020511F0020F407002017
S31900008980FEB50D0012214843B4490C186B460122972120781A
S3190000899400F024FA68460088FF21090201402943684601807E
S319000089A80A469721207800F003FA2089019002AB0122217984
S319000089BC207800F00FFAA74D474E684600892900014048029C
S319000089D021786C225143711848310A8829001140FBF7BBFE19
S319000089E4691C884200D3280085B20198A84200DA85B2207CC8
S319000089F80127410839420ED101995E398D4202D3A17A092978
S31900008A0C04DB02210143217400205EE0491CA172F7BD914812
S31900008A20305C38424FD1FF265636A07A092819DB8A48406AAA
S31900008A3400794008384204D1A8190199884215D341E02800C2
S31900008A482230019988420FD3FFF783F88149896AFFF782F8DE
S31900008A5C82490978814232D3A07A002802D1A02636010CE0EE
S31900008A70A07A032801DACB4E07E0142802DAC026B60002E036
S31900008A84202800DAAB36E0898019E081A189019A8918491BA8
S31900008A98A18180B289B2884211D3A07A3B2815DB00AB9B1CB8
S31900008AAC01226179207800F095F968464088A1788907890FE6
S31900008AC0C840384201D0002100E00121200000F00DF8F7BD5D
S31900008AD4401CA072F7BD00006D8C00006C0500005015002077
S31900008AE88C020020F8B504000E006B460122A321207800F0E7
S31900008AFC71F9A178A94F01256846008801228A4010426ED00C
S31900008B10002E6CD00023E2782078FEF7F1FDA07886083220F1
S31900008B24464308366B460122F1B2207800F056F903200121DD
S31900008B38A2780323134008339940227C93082B426A4612888C
S31900008B4C03D08A4369460A8002E011436A4611800121A27883
S31900008B60032313401B1D9940227C13092B426A46128803D02D
S31900008B748A4369460A8002E011436A4611800121627810401E
S31900008B880C308140E0780228684600880BD1014368460180CF
S31900008B9CA07821786C22514379180818A13005700BE088433F
S31900008BB069460880A07821786C22514379180818A1300021FE
S31900008BC4017068460288F1B2207800F0F3F86B46012221796A
S31900008BD8207800F001F989206178724A5054207C0821014316
S31900008BEC2CE06B460122A121207800F0F3F868460188A27809
S31900008C00012090408143684601800288A121207800F0D2F8D8
S31900008C14A07821786C22514379180818A13000210170A07847
S31900008C288540AAB2A521207800F0C2F86078FEF702FD882095
S31900008C3C61785B4A5054207CF72101402174207CFE21014076
S31900008C50217402212078FEF721FCF1BD30070020FF030000A1
S31900008C64010A0000BC180000F8B5FEF7BDFF4F4F38784F4DCF
S31900008C78002808D11022A221102000F099F8FEF768FFA862D5
S31900008C8C86E0052801DA04260CE00A2801DA152608E01428DE
S31900008CA001DA2B2604E0192801DA552600E062260124287CE2
S31900008CB4204203D031000020FFF760FE2220285C204203D0D1
S31900008CC831000120FFF758FE287C204262D122216A5C22424E
S31900008CDC5ED1C00820423FD0A97928780326D30801221342D8
S31900008CF06B4626D000F074F80120A978314008318840694604
S31900008D040988814308436946088068460288A979287800F094
S31900008D184FF86B460122297EA87C00F05DF8287D06400836ED
S31900008D2CB44068460088A0430443684604800288297EA87C52
S31900008D400EE000F04DF868460088A9780E400836B440A0433C
S31900008D546946088068460288A979287800F02AF80A24287CF0
S31900008D680A210140022902D16878FCF707FB2220285C0440A8
S31900008D7C022C02D1E87CFCF7FFFA2022A221102000F014F85B
S31900008D90FEF734FF00210220FCF719F93878401C3870F1BDF7
S31900008DA455050000501500208C0200200308002030070020A6
S31900008DB81CB501AB4000012404431C7059706846028000787B
S31900008DCCD8706846407898700122042101A801F0FEFC13BD2B
S31900008DE0F0B587B015001F0004AA40001070517095701E48CF
S31900008DF4D070FF2010711D4E8024640274600C2000E000BF71
S31900008E08401EFCD102AA052104A801F018FD02A8C278017943
S31900008E1C0906090C0A433A80022D06DBB81C0200691E490655
S31900008E30090E01F008FD6D2000E000BF401EFCD134606B467F
S31900008E440DE0410079180A889A806A4612795A7001AA52782F
S31900008E581A706A4612880A80401CA842EFDB07B0F0BD00002E
S31900008E6CFFFF000004F10F400100724805224823C35C8B4271
S31900008E8003D05830521EF8D10020704780B5FFF7F1FF00282A
S31900008E9408D001886A4A914204D15521415C002900D1018079
S31900008EA801BD10B50C00FFF7E1FF048010BD0020BF49820050
S31900008EBC8A18926E002A0CD0CB68934209D01388002B06D176
S31900008ED04923D35C002B02D0CA6001207047401CC0B20528F3
S31900008EE4E9DB0020704710B5544A05234924145D002C0BD168
S31900008EF84823D1545421505400201080B248C260012049324F
S31900008F0C107010BD58325B1EECD1002010BDFCB5484A0020EE
S31900008F200023AB499C000C19A26658325B1C052BF8DB8300D0
S31900008F34CA180192926E08321CD0421C0C006834E3180093F4
S31900008F4811E09300CB189C6E250008350AD0009D2D685426B6
S31900008F5CAE5D5427E75DBE4202D2009E34609D66521C052A8B
S31900008F70EBDB019A926ECA60401C0428D9DBF3BD38B52F4D07
S31900008F84DC22520000212800FBF7FCFD894C14220021200003
S31900008F986830FBF7F5FD0922002158342000FBF7EFFD00204D
S31900008FAC254958224243A952401C0528F9DB31BD00B5B3B0E0
S31900008FC0FCF714FA6846C7306946401A33B000BD00B58446C9
S31900008FD4FFB0B0B06046FEF7D7FD7D4869460818401A7FB0E8
S31900008FE830B000BD00B5844679488544604601F0B7FF7848BC
S31900008FFC69460818401A77498D4400BD00B5844675488544DF
S31900009010604602F0F9F8744869460818401A73498D4400BD8E
S3190000902400B58446714885446046FDF76FFB704869460818A6
S31900009038401A6F498D4400BD08000020FFFF0000F8B5FFF7B5
S3190000904C99FF74210A20FFF74AFF584E30005430009030005A
S319000090601030FEF7FFFD0099087000980078002803D1FFF7B2
S31900009074ADFF002847D063210920FFF734FF30001030FEF7BC
S31900009088EDFD0099087000980078002803D1FFF7C5FF0028E5
S3190000909C35D064210820FFF722FF30001030FEF7DBFD00991B
S319000090B0087000980078002803D1FFF77FFF002823D06E2104
S319000090C40720FFF710FF30001030FEF7C9FD00990870009892
S319000090D80078002803D1FFF785FF002811D070210620FFF7DA
S319000090ECFEFE30001030FEF7B7FD009908700098007800280C
S3190000910005D1FFF781FF002801D10020F2BDFFF704FF341DF6
S319000091140020A0600099487330001030FEF7A0FD00990870BA
S319000091280098007800283ED1A06800280CD0FEF710FDA168CF
S3190000913CC96CFEF70FFDE064A068E16C026D914200DB0165C7
S31900009150FEF703FD05002168FEF702FD2560002817D00021D9
S319000091648A00B218926E002A0ED0A36893420BD013881D0022
S31900009178204FBD4206D0854201DA002301E005005B1B1380E5
S3190000918C491C0529E8DBFFF790FE002808D0FEF7DEFC01001F
S319000091A0A068C16401210830FEF768FDA0600098407B002859
S319000091B4B2D0F2BDB804002080B5FFF759FE002801D0008891
S319000091C802BD0C4802BD0000B8040020BB020000B4FBFFFF75
S319000091DC4B0400004C040000BCF9FFFF3F0600004406000098
S319000091F0CCF7FFFF3308000034080000FFFF0000F1B592B047
S3190000920409AB0122962112A80078FFF7E7FD12A804780E2052
S319000092186043C04909186846808C8005800D0A7B52008852F2
S3190000922C0A7B521C0A730126D2B2062A05D14A7B002A00D147
S319000092404E7300220A736C226243B54B9A1808924832009229
S31900009254FC252D024A7B002A13D0002000225300CB5AC0184C
S3190000926880B2521C062AF8DB00990F882F40C01C0621FBF7B5
S3190000927C6BFA8005800D384303E0009909882940084300998C
S319000092900880009800888005800DCF4940180D2811D3CE486B
S319000092A4610009199D4A511808180178FF2901D0491C017075
S319000092B8009800880540700228430099088003AB9B1C0122B1
S319000092CCA42112A80078FFF785FD6846C0890009C049087098
S319000092E0062044438E480019807880090A9000250795019566
S319000092F426E000200599088007980599098849084018079006
S319000093080698408A8005400B009909888905890DFBF71FFABA
S3190000931CB102884200DB481E059908820698428A0499C9B2CF
S3190000933012A8007800F0F6F8641C042C43DB0198401C0190BF
S3190000934401980A99884200DB90E00BAB0D22014632204143BC
S319000093580931C9B212A80078FFF73EFD0198800069460873A0
S3190000936C29006846858D007B85400D43ADB20198002821D15C
S319000093800BA8C088009948814002009909888905890DFBF7F4
S31900009394E2F9FF2800DDFF200099488100984189BB4848436F
S319000093A8BB30BB214900FBF7D4F9B949401A00B2401D0A2146
S319000093BCFBF7CAF900B2029000246846007B0019C0B2049032
S319000093D04000089908185E30059060000BA9081806904089CC
S319000093E4010486D504992A00CA40D107F9D58004800C070081
S319000093F85621049A089B9A18515648433D307A21FBF7A4F928
S3190000940C381A80B2522826DBA149049A0A235A43A04B9A1858
S3190000942051188A88029B002B01D5521C02E0472B01DB521E0B
S3190000943492B24243CB88D21A0B88434343434888471E012021
S31900009448B84018184B88D840121A0889431E012098401018B8
S3190000945C0989C8404AE7FA218900484331034018400B43E7FB
S319000094700BA88088009908814002009909888905890DFBF783
S319000094846AF9B102884200DB481E00990881009800895821F1
S31900009498009A515644181481A4B22200C82189014808029BB0
S319000094AC1A2B08DA1923029E9B1B5A431018FBF74BF92018BA
S319000094C005E0193B5A431018FBF744F9201A009908810BA856
S319000094D40089009988814002009909888905890DFBF739F99F
S319000094E88021C900884200DB481E0099888100984580C148ED
S319000094FC4168009A1289891841600799009A51600168009A48
S3190000951052688918016013B0F0BD0000AC03002050150020C1
S31900009524F1B582B00E006846007A6C214843B4490818019059
S31900009538B00001990D1880352868D10A084328600124C008CA
S3190000954C204004D031006846007AFEF71FFA2878C006C00E36
S31900009560022837D1019881190220C043A1228A5C002A2CD098
S319000095740122A9310A70296808402860B5082F000A3F6B461F
S31900009588F9B26846007AFFF727FCB607B60F700080196946A3
S3190000959C098807228240914384400C43684604800288F9B2EB
S319000095B0007AFFF701FC6B46012232204543A9191231C9B206
S319000095C46846007AFFF70AFCF7BD296808402860F7BD0000A0
S319000095D806FEFFFFDF090000381B002090B587B08648874902
S319000095EC415C0E2211424CD101A90022002300241CC1002117
S31900009600824A82180092009A12880123A3401A4213D00022BC
S3190000961401AB1B196C276743C719BF18A9373F78002F05D0CD
S319000096281978012797400F431F700121521C082AEEDB641CAC
S3190000963C0C2CE2DB002924D00022A1211020FFF7B5FB002226
S31900009650A2211020FFF7B0FB0024009800880121A1400842DB
S3190000966405D001A8025DA121E0B2FFF7A3FB641C0C2CF0DBA4
S319000096780822A2211020FFF79BFBFEF76AFA624908600120A2
S3190000968C00E0002007B090BD521C0000D20A0000CE020000A6
S319000096A028150000D0B58AB000275A4800880121B9400842FE
S319000096B400D19CE0002001906C207843504908180390483093
S319000096C802900EE008688022520202430A60002005990870BD
S319000096DC641C042C1DDB0198401CC0B2019001980621794358
S319000096F0444A51188978890988427ADA32214843049006AB95
S31900009704042201461231C9B2F8B2FFF767FB0022A221F8B28F
S31900009718FFF74EFB0024019880000619F6B203988019A930E7
S3190000972C059000780028D3D0600006A9085A8005400B02996F
S3190000974009888905890DFBF708F88021C900884200D3481EFB
S31900009754B100039A5118803180B2FF2218329042B2D3F800A7
S319000097682B4A1018805D00283BD00120B04069460880684644
S3190000977C0288A121F8B2FFF719FB1022A221F8B2FFF714FB2F
S31900009790FEF7E3F90600FEF7E0F93100FEF7E0F90228F8D326
S319000097A42022A221F8B2FFF705FB00AB9B1C012204990931AA
S319000097B8C9B2F8B2FFF710FB684640880121A140084207D0D7
S319000097CC02984088694609880143029841807CE70F484078D0
S319000097E0202101430D48417075E70868802212026FE77F1C71
S319000097F40C2F00DA57E70AB0D0BD0000B41A0020501500204E
S31900009808010A0000E4050000F0070020341B0020CC010020DF
S3190000981CE424002010B55D4C5D49096841430800FA21890055
S31900009830FAF793FF60805A48027861885300C3189980521C01
S319000098440021D2B2102A05D14278002A01D1012242700022A8
S3190000985802706288A388934201D2D31A00E09B1A9BB2652B68
S3190000986C0CDA4378002B09D000224B00C3189B88D218491C83
S319000098801029F8DB08321209A28010BD38B545480188C82093
S319000098944843AA30FF215631FAF75DFF040080B2FFF7BCFF7A
S319000098A83B4A51883E4B5888002588420DD255811978491C45
S319000098BC1970C9B2032905D1A1B25288101A80B200F005F816
S319000098D031BD401A50811D7031BDE0B582B00200FA20800087
S319000098E45043FAF738FF00902F4E30483018017801220A43F9
S319000098F8027000252D4F785DFF2809D0694600F019F8009826
S3190000990C002814D06D1CEDB2042DF2DB0025972000017119A8
S31900009920085CFF2809D0694600F008F80098002803D06D1C0E
S31900009934EDB2602DEFDBE3BDF8B51B4A1D4B1418E5182B783D
S319000099481C0901231B4E965BE6401E421ED02D782E07360FCF
S3190000995C6C277C4314194A342488F4401C4213D073002C092B
S319000099706C256C431219D2185E3212880B689A4201D29A1A88
S3190000998402E00022074C22700A600721FDF79AFDF1BD000015
S3190000999830F2FF1FAC1A002088070020A81A0020F8070020DF
S319000099AC50150020010A0000F40700206C050000E40500009C
S319000099C010B58AB003A81821FDF734F9684600BF3CA11CC95A
S319000099D41CC0344C0C2269469D2000012018FDF787FE182297
S319000099E803A930482018FDF781FE80202E49086000F011F81E
S319000099FC00F018F80AB010BD2B4820214160402242605023FE
S31900009A1000BF5B1EFCD1026000BF0160704780B5002218216E
S31900009A24244800F0D8FEFFF7EBFF01BD38B500241C4D214875
S31900009A38285A0121A140084216D06B460122A9212000FFF7AB
S31900009A4CC9F968460088FF21090201409D2000012A19105C2F
S31900009A600143684601800A46A9212000FFF7A4F9641C0C2CF4
S31900009A74DFDB31BD10B5114C2078002804D0012805D0032851
S31900009A8806D010BDFFF7C7FF10BDFFF7CDFF10BDFFF7C1FF53
S31900009A9CFFF7C8FF0420207010BD000050150020CC0500001C
S31900009AB088F00F4084F00F401C1B0020E40500002C1F002067
S31900009AC4FFFFFFFFFFFFFFFFFFFFFFFFE0B58EB0060030216A
S31900009AD801A8FDF7ABF830002EE00021274A284B5B189D5C85
S31900009AEC2A07120F4B00264FFF5A012383401F421BD0009230
S31900009B00009200239B189B085F00BC462D09AF0001ADED1946
S31900009B146746ED192F889B00D31A4210920F121892109200F4
S31900009B28821A92009B1801229A403A432A80491C6029D3DB82
S31900009B3C401CC0B20025311D8842CCDB114800880121A94071
S31900009B5008420CD0A80001A90F183A880121E8B2FFF72AF9C5
S31900009B647A883321E8B2FFF725F96D1C0C2DE9DBB208A621DC
S31900009B781020FFF71DF90EB0E0BD00BF6C0500005015002087
S31900009B8CEC020020341B0020F0B58BB0FDF752F803246F4846
S31900009BA000909C26B60001AD0098FAF76BFF002822D16B4F2D
S31900009BB4381D0A90AE8001A8801D69491E22FAF7EBFF310036
S31900009BC8381D00F02EF80190092201A9009801F000FCA888FD
S31900009BDC82080A99C64801F0FAFB01A800F009F8002801D0BB
S31900009BF0012002E0641ED7D100200BB0F0BD10B5564C0068D7
S31900009C04216888420BD1201D0188C14A914206D22000243027
S31900009C1800F007F82168884201D0002010BD012010BD10B57F
S31900009C2C02000023002002E0D45C00195B1C9BB28B42F9D351
S31900009C4010BD0000F8B5132216A1B348FDF752FD434D9C2119
S31900009C548900281DFCF7ECFF3F4C1E22A11D4048FDF705F947
S31900009C68002813D1261D3088A84988420ED227002437014677
S31900009C7C3800FFF7D4FF2168884205D132883900281DFDF778
S31900009C9031FD03E000F0BCF8FFF77CFF00F0C3F82870F1BDA3
S31900009CA47265636F766572795F706F655F64625F6B657900C7
S31900009CB8F8B5B14D9048008896496852A82252009549964816
S31900009CCC2818FDF711FD00243020604393490F1806223900C1
S31900009CE03231924806236343EB181818FDF702FD0A2060436B
S31900009CF42E180A224437390030003A30FDF7F8FC102C08DA90
S31900009D080A22200114490918091D87483018FDF7EDFC0C2C24
S31900009D1C0BDA6000001903229749984B1B185918974B281821
S31900009D30C018FDF7DFFC641C302CCBDB2022944994482818B5
S31900009D44FDF7D6FC2022934993482818FDF7D0FC00F097F8C7
S31900009D58F1BD000000F4000054FBFF1F2B150000F8B56B4D3D
S31900009D6C6B48285A634908808A4EA82252006A4829189220DB
S31900009D8040003018FDF7B6FC00243020604366490818009025
S31900009D9406226548062161436918091800983230FDF7A6FCE3
S31900009DA80A2060432F180A2239003A3100984430FDF79CFC25
S31900009DBC102C07DA0A225B48391820013018001DFDF792FC48
S31900009DD00C2C0BDA6000001903226C492B185918684B694FEA
S31900009DE43818C018FDF784FC641C302CCBDB20226748291815
S31900009DF86548FDF77BFC2022664829186448FDF775FC0220D5
S31900009E0C3070F1BD10B5634C9C2292006249201DFDF76AFCE8
S31900009E200120607010BD38B500F06CF83A4D6969814206D037
S31900009E3400BA814201D10C2032BD032032BD1E22584928008F
S31900009E481A30FDF712F8002801D0042032BD686900BA686158
S31900009E5C00246B4601226C212000FEF7BBFF68460088382109
S31900009E70695C884201D1082032BD641CE4B20C2CEDDB0D201D
S31900009E8432BDF0B583B000263C4F38001A3045491E22FAF70B
S31900009E9881FE380014300090424800998880FDF758FE0500AB
S31900009EAC6D1CE8B2F221FAF74FFC491C38203954002401AB10
S31900009EC001226C212000FEF78BFF38203A5C684680888242D1
S31900009ED403D0641CE4B20C2CEFDB761CF6B2032E01DA0C2C0B
S31900009EE8E0D06C211020FEF763FF00F007F800990860F7BDF8
S31900009EFC24F40000361B002080B5AF21C900294800F012F88A
S31900009F1002BD0000DD030000541F00206A05000078FCFF1F04
S31900009F243A03000030F2FF1F1A0200008A04000080B50022A5
S31900009F3800920A000100002000F005F80422694600F001F8A7
S31900009F4C02BD70B513005A1E002B12D00B78491C0824050066
S31900009F6040001E0602D5060001203043002D02D505001048B1
S31900009F7468405B00641EE9D0EFE770BD541F0020DD09000019
S31900009F88501500206C050000E00600204A050000C00600208E
S31900009F9C2A05000054FBFF1F4C1500002B1500007C050000ED
S31900009FB06C1F0020B71DC10410B50400FCF73EFA4021324884
S31900009FC402680A4302603148002282706300037042724271A0
S31900009FD88171C2710A210172810D2C4A11608178C0220A430F
S31900009FEC8270FCF72DFA10BDF8B5284C6078617802220A433F
S3190000A000627001210025102210420BD0637810261E43667086
S3190000A014214B1B685E78082737435F70012600E00026EF23B6
S3190000A028470606D5400720780BD5024322706A460FE0002E93
S3190000A03C25D12678164213D0014006D0207803402370A0789E
S3190000A0506946087017E06A4601210020FCF727FE002801D1D4
S3190000A06468460578A5700CE0A078694608700020FCF75DFE09
S3190000A078002804D00848017820220A430270FCF712FBF1BD5A
S3190000A08C348004400060064000E100E00260064024F2FF1F7F
S3190000A0A0E424002070B50500FCF7C8F946480168020D0A434D
S3190000A0B40260454C0026E670A6700E20A071B7208004290149
S3190000A0C8FAF747FB8104C90E217060700F20A072E67226725D
S3190000A0DC6672217901432171C02162790A4362718022520151
S3190000A0F0374B1A60E2780C231343E37062791143617121798D
S3190000A10408432071E079E07820210143E170FCF79BF970BD2A
S3190000A118F8B52E4801684A78022313434B702C4C4025802725
S3190000A12C0F266178890615D521796A4611706178314204D0A7
S3190000A14000684178394341700AE069460020FCF7F0FD0028F6
S3190000A15404D02148007828431F490870607828421AD020782D
S3190000A168284217D06A4600210020FCF79CFD0021C943884218
S3190000A17C09D0002803D12078BF2101402170684600782071F3
S3190000A19004E012480078074310480770607806436670A078D7
S3190000A1A4C0210143A170F1BD4021002801D1094800E00A48DF
S3190000A1B802780A4202D1027811430170704700003480044006
S3190000A1CC00A0064000E100E024F2FF1F03A00640E42400208D
S3190000A1E003B00640774800210122774B1B781B071B0F052B98
S3190000A1F400D9704710B501A4E45CA744041018202830007810
S3190000A208042815D000F078FA10BD017000F07AF810BD0170EB
S3190000A21C00F0D6F810BD017000F04AF910BD027000F078F959
S3190000A23010BD027000F0C6F910BD9E480078002800D170474B
S3190000A24470B59C4E182255213000FAF79BFCFFF7E4FBFCF7C1
S3190000A258F3FCFA25AD00AD4C21002800FDF7E6FC1822AA2114
S3190000A26C3000FAF78BFCFFF7D4FB21002800FDF7DBFC70BD2A
S3190000A28080B530214143A44A511844310978F8F749FE00F047
S3190000A29401F802BD0100A0480278012004291BD91F3913D018
S3190000A2A8491E13D00B3915D0891F0DD0491E0DD0891E09D0E0
S3190000A2BC091F07D0091F032906D90D3904D0491E012904D8CF
S3190000A2D0104070475108084070470020704780B5FDF73BFCDE
S3190000A2E48D490A78830502D50223134301E0FD2313400B705F
S3190000A2F80A78400502D50120104301E0FE201040087001BDB5
S3190000A30CF0B587B000240025009401A81821FCF78BFCA84832
S3190000A3200078800701D5FF2000900C27FFF7D7FF5F2606E035
S3190000A334302E04DAF0B2FFF7A1FF204304006D1CEDB2082DD7
S3190000A34808D100986040FFB201A9C8557F1C0025002400E0AE
S3190000A35C6400761EE8D55EE080B5302141436B4A5118443157
S3190000A3700978F8F7D7FD00F001F802BD04281CD91F3818D087
S3190000A384401E12D00B3816D0801F12D0401E0CD0801E0ED01F
S3190000A398001F0CD0001F032805D90D3803D0401E012804D90C
S3190000A3AC07E05B480078800703D50220704701207047002065
S3190000A3C0704700002C1F00203CFDFF1FF0B587B000240025E5
S3190000A3D40094002701A81821FCF72AFC77480078800701D525
S3190000A3E8FF200090FFF777FF5F2606E0302E04DAF0B2FFF701
S3190000A3FCB3FF204304006D1CEDB2042D08D100986040FFB213
S3190000A41001A9C8557F1C0025002400E0A400761EE8D501A908
S3190000A4240A20FAF76FFD07B0F0BD70B505002E000124302066
S3190000A438704337490818443001782800F8F76EFD04281ED925
S3190000A44C1F3813D0401E14D00B3818D0801F0DD0401E0ED097
S3190000A460801E09D0001F07D0001F032807D90D3805D0401ED3
S3190000A47401281BD82848007802E02748007840080440200055
S3190000A48870BD04212800F9F7B9FF00280AD090204000B100F5
S3190000A49CA44A5118085A8009204201D0022070BD012070BD94
S3190000A4B0002070BDBD1800001C1B0020F0B587B000240025F4
S3190000A4C40094002701A81821FCF7B2FB62480078800701D5C2
S3190000A4D8FF200090FFF7FFFE5F2606E0302E04DAF0B2FFF789
S3190000A4ECA0FF204304006D1CEDB2042D08D100986040FFB235
S3190000A50001A9C8557F1C0025002400E0A400761EE8D586E754
S3190000A514416C000030F2FF1FEC070020F0B587B00C22FF2103
S3190000A52803A8FAF72DFB002403AF01AE347001A8F9F778FD1E
S3190000A53C002839D0302060434649081844300090012501788F
S3190000A5502000F8F7E7FC01281DD9801E06D0293828D100987A
S3190000A56440794009284214D0707838180378704A9446B2781C
S3190000A5786F4989186246895C0A07120F012191408B4303707D
S3190000A58CF07838180178337905E0707838180178654B9C46B0
S3190000A5A0B378654AD2186346D25C1207120F9540A94301709A
S3190000A5B4641C302CBCDB03A90E2032E73BFDFF1FD0B588B014
S3190000A5C80C22FF2103A8FAF7DBFAFFF784FE0024574F03AEC7
S3190000A5DC6846047101A8F9F723FD00282ED02000FFF71FFF2F
S3190000A5F0010052486200524B9A181218C80712D51078602815
S3190000A6040FDA4B4B3818C05C0309F31800931B789C46030728
S3190000A6181B0F01209840634683430098037088070ED5507851
S3190000A62C60280BDA40493818405C010971180A7803071B0FE9
S3190000A6400120984082430A70641C082CC6DB03A90E20FAF7A8
S3190000A65459FC08B0D0BD00003BFDFF1F30F2FF1FFCB50020EB
S3190000A66800210022354B9D7B01241F7E0526374203D10121A1
S3190000A67C25439D7302E0FE262E409E732F4D00951D8A009E71
S3190000A69036882E4001962D4D2D78019E009F7F883E4201D038
S3190000A6A4254202E0009FBF883E4200D001228024264E367834
S3190000A6B87607760F06D0022E14D005D3042E11D014D314E0D6
S3190000A6CC080012E020480078C207D20F012048401043E90704
S3190000A6E0C90F084209D11C480460F3BD188B0006C00F00E094
S3190000A6F410000028F5D017484460F3BD10B58AB003A81821B9
S3190000A708FCF794FA684600BF13A11CC91CC069460E20FAF706
S3190000A71CF5FB03A90A20FAF7F1FB03200C4908700AB010BD09
S3190000A73058FBFF1F6C05000050150020A303000028150000C5
S3190000A74430F2FF1FC2FDFF1FEC07002040FDFF1F381B0020FD
S3190000A758C4F00F402C1F0020FFFFFFFFFFFFFFFFFFFFFFFF85
S3190000A76C802040023E4908602020803908603D480168802211
S3190000A780D2030A4302603B481C21017000214170C171512194
S3190000A79481704021C2780A43C270027811430170704710B5E5
S3190000A7A833498A78334A20230C781C4204D1401C9042F9D3A8
S3190000A7BC012010BDF8248C700C781C4204D1401C9042F9D3CC
S3190000A7D0022010BD8878002010BDF7B523492022D3026846B6
S3190000A7E4007A002801D04B6001E024484260214C20781042F7
S3190000A7F8FBD00C200C2500E000BF6D1EFCD107E0009E765DD0
S3190000A80CA670202627783742FCD06D1C6E463679EDB2B54270
S3190000A820F2D36D2400E000BF641EFCD16C46247A002C01D08D
S3190000A8340B6003E080390A6000E000BF401EFCD1F7BD30B536
S3190000A8480B4B9C781C78A406FCD5002407E0055D9D701D786E
S3190000A85C2D06FCD59D781555641C8C42F5DB30BD04F10F4010
S3190000A87034800440006007400360074051C3000084F00F40AE
S3190000A88480B56E20FEF700FB01BDF0B585B0002502AC7748DD
S3190000A898405D00903021484375490E1844363078694608716F
S3190000A8ACFF21EC31009A5200714B9A18575C032866D10120C5
S3190000A8C0317A4908014261D06B49098B490A01425CD10522DC
S3190000A8D4002102A8FAF756F92770FF20A070032071794A083A
S3190000A8E8032111406278FC2313400B4363700029194610D00C
S3190000A8FCEF230B4090225200944600998A005C4989186246F6
S3190000A910895A0906C90F09011943617002E0EF220A4062701D
S3190000A9242279FD211140554A12789308022213400B432371F2
S3190000A938184008210143217102A90220FAF7E0FA96229200CC
S3190000A94C02214D48FAF772FB70794C49C95D89290DD1202166
S3190000A960014371713079802108401521014331710420307045
S3190000A9740122092104E0DF2101407171092203210098C0B21C
S3190000A988F9F788FB01233278684601790098C0B2FCF758F8FF
S3190000A99C6D1C302D00DA78E70020FAF783FA05B0F0BDF8B5E5
S3190000A9B000203249802230234343C24CE318009344331C79CF
S3190000A9C414401C7101241D78203D04D06D1E06D06D1E0C2D88
S3190000A9D836D89D796D09254232D1F5256D0046008E1975195F
S3190000A9EC2E78FF2E1DD06D78FF2D13D090256D0086008E194E
S3190000AA00755BAE0926420BD01F7A274220D19E79770927427F
S3190000AA141FD01C79102525431D7106E09D796D09254222D1AD
S3190000AA281D792C431C711C7914431C715C79E72525405D71F5
S3190000AA3C07245C700023009C24342370401C3028B3DBF1BD6F
S3190000AA501C790D25E1E7F42676008E5D3709274202D12D0930
S3190000AA64AD07DFD01C790C25D5E71C790325D2E70007002056
S3190000AA7830F2FF1F58FBFF1F3DFDFF1FDC0700208C0200200A
S3190000AA8CF1B586B00522002104A8FAF777F8FF2004AC207021
S3190000AAA0A070032320790321014021710025002200219020BE
S3190000AAB440006E46367EB600824FBE19301803906846007E7B
S3190000AAC8302670437D4E3018483000907D4802900127009839
S3190000AADC00784006400E401E11280DD801A6365CB74400BFE5
S3190000AAF0122A5A5E726A72EEEEEEEE16161C2A587262012291
S3190000AB046BE00122022168E0039800880006000F03210140C1
S3190000AB18891D039800880006000F03220240D21C694E02989F
S3190000AB2C407A8008384207D00298C0790340581E8041C00F60
S3190000AB4030704CE035704AE00A21092247E00B2245E0E07839
S3190000AB5404250543E570607804250543657000984078450866
S3190000AB6803202840FC2566782E4006436670E67835400543A1
S3190000AB7CE570029D2E783E42257902D02F43277102E0FE2625
S3190000AB902E402671EF2500280DD0039800880006C00F000194
S3190000ABA466782E4006436670E67835402843E07005E06078E1
S3190000ABB828406070E0780540E5702579FD202840029D6D79B1
S3190000ABCCAD0802263540054325712B40042018432071F520AF
S3190000ABE040006B461B7E5B00374DEB181818057840786B46D9
S3190000ABF418719048FF2D07D04319009E3678F60901D01A70E1
S3190000AC0800E019706B461B79FF2B07D0C018009B1B78DB0999
S3190000AC1C01D0017000E0027020798008012825D1009800783A
S3190000AC304006400E072803D101A91220FAF764F90098007839
S3190000AC444006400E112801D0122819D100980078C00911D179
S3190000AC58A5706846007920707648774989788A005118764AE4
S3190000AC6C5118081804A90522F9F792FF07B0F0BD6846007965
S3190000AC80A07003E000980078C009E6D02570E7E710B504000C
S3190000AC94FF2813D0022808D108798208012A04D18007800F78
S3190000ACA8082202430A712000FAF72AF9962292002100A84819
S3190000ACBCFAF7BCF910BD000030F2FF1F58FBFF1F38FDFF1F07
S3190000ACD0481B0020E0B584B0070030207843A0490818009073
S3190000ACE4483000784606760E009924310191534D31001BD05A
S3190000ACF8711E20D0491E26D0491E01292FD9891E022968D9BA
S3190000AD0CC91E03290ED9091F012949D9891E18D0491E1AD0DF
S3190000AD20491E20D0491E012959D9C91E062971D880210840B7
S3190000AD340643009848300670EFBD0121380000F085FB0600BA
S3190000AD48022E64D135E0380000F092FC21E0380000F08EFC0E
S3190000AD5C0600032E59D1042657E0E878012854D128790028A4
S3190000AD7051D102A9380000F0EBFE00280FD00198807C032824
S3190000AD8406D0764880890199498C401873498881380000F064
S3190000AD98E7FF06003BE06846027A05213800F9F779F933E09D
S3190000ADAC3100380000F04EFB0600022804D16879022829DAD8
S3190000ADC0401C0AE00E2801D00F2824D16879002802D01A26E5
S3190000ADD4522000E0022068711BE06148A9788A005118174AFF
S3190000ADE85118081801788907890F10220A430270380000F00E
S3190000ADFC97FD019908703100380000F01FF80600A878401CA5
S3190000AE10A87000E01A26FCF7A0FE0199C86100984830007814
S3190000AE24802108407106490E0143009848300170EFBD0000EC
S3190000AE382C020020E9050000E4070020501500207BB583B0D1
S3190000AE4C481F012807D9801E03D00A38012804D905E00925B0
S3190000AE6004E0082502E0142500E00D466846007B3021484374
S3190000AE743A49081800906846007C0026052801D0112818D121
S3190000AE8800982430807C03280FD100982430C07B8007800F80
S3190000AE9C032801D1002200E0012208216846007BF9F7F6F84A
S3190000AEB003E06846007BF8F7D7FF009824300078072848D10B
S3190000AEC40098443000786946087168460479302C0FDB09222C
S3190000AED80321007BF9F7DEF8009924310E7084480078400605
S3190000AEEC29D400984430468025E0009844308079800607D511
S3190000AF001224012207216846007BF9F7C7F818E06846007CBC
S3190000AF14052806D0072802D0112802D00FE013240DE0009869
S3190000AF2844304079C006800F04D0022804D004D2112402E0CE
S3190000AF3C102400E014240098443004700123220068460179C1
S3190000AF50007BFBF77BFD280006B070BDDC07002030F2FF1FB4
S3190000AF64ED050000F8B56448C0680830FCF778FE624908709C
S3190000AF780878002800D1F1BDF9F790FD00280BD1F9F780FCAB
S3190000AF8C08E0641CE4B2302C00DAA3E05A49887101200870BF
S3190000AFA05948017804220A4302705448C0685749018008307B
S3190000AFB4FCF756FE51490870087800283CD000204F49086056
S3190000AFC888805148008B514901404F48018300210B20F9F711
S3190000AFDC95FF0120F9F766FFFAF7C6F8F9F79DFCF9F704FD28
S3190000AFF0FFF74DFCFFF7DBFC002745498F810120694608702E
S3190000B0040CE00024FFB2390006294BD801A2525C974400BFFB
S3190000B018080C325E66868A00002510E03548C0680A2101809E
S3190000B02C0830FCF719FE334908700878002803D102213648B7
S3190000B040FCF71CFE0125354C2EE0FAF793F83049098B022881
S3190000B05403D180208000084303E0002803D12F4808402A4992
S3190000B0680883FF25012025494870C87018E0234A14712A4943
S3190000B07C05E021490979012909D127491E4A927893009A18BE
S3190000B090254B9A185418022506E0FF2504E0062502E01125C0
S3190000B0A469460C7000262048805DFFF7EDFC761C302EF8DB5A
S3190000B0B821002800FFF7E8FD00241A48005DFFF705FE641CFE
S3190000B0CC302CF8DB7F1C68460078002895D1012000240C4A51
S3190000B0E0302161435118483109784906490E1A2900D04CE712
S3190000B0F400204FE73DFDFF1FB80400200C050020E40700207C
S3190000B108FC070020FFFF000030F2FF1FFFFE0000C8040020E3
S3190000B11C2C020020FFFD0000E9050000501500200007002035
S3190000B13080B5FBF785FD914800210170417081708F48017007
S3190000B144FBF751FC00218E48FBF7EEFB01BD01208C498D4A55
S3190000B1588A5C1209024200D0704730B583B000226C462260A3
S3190000B16C884BC9184B8809885940874B0C00D440044028D0EA
S3190000B18001249440DD78AD08054205D06D466D882C436D46CC
S3190000B1946C801CE01D782D09054213D07D4800688178042278
S3190000B1A80A438270FBF748FDFA204000FCF733FDBFF34F8F0A
S3190000B1BC774878490860BFF34F8FFEE76D462D882C436D4692
S3190000B1D02C80521CD2B20C2ACEDB68464088002805D000A9CC
S3190000B1E4891C0C20F9F78EFE37BD68460088002807D069462C
S3190000B1F80D20F9F785FE8020C000FBF70DFC37BDF0B583B076
S3190000B20C6548C0680830FCF727FD644908700878002800D166
S3190000B220ABE0FBF7D3FA554F0126FCF796FC01905E480078CB
S3190000B234082101435C4801705C48047805210D20F9F764F8BF
S3190000B248594908700878844202D00020F9F7EEFC55480078AB
S3190000B25C4000554909180920F9F750FE00F05AFF01F0F8FC44
S3190000B270F8F7FBF950480078002806D0454800784009304213
S3190000B28401D0FBF7A7FD7878401C7870C00701D4FFF75DFF27
S3190000B29878780A21F9F75AFA002907D101F01AFDF8F720FD28
S3190000B2ACF9F7A4FC01F058FD7878000701D1FBF787FA002452
S3190000B2C07878F02800D17C7038780C2802D00D280CD012E0F6
S3190000B2D4FBF789FB00212A48FBF726FB002200218020F8F772
S3190000B2E8D9FE1FE0FCF735FC0090BE70FFF7C6FA18E0B878B6
S3190000B2FC002815D00025FA21C9000098FCF733FC002806D06A
S3190000B31001252A48407810210143284841702848007805430D
S3190000B32402D00A203870BC703878401C3870FCF712FC0199F0
S3190000B338FCF712FC01001948C0681E2909D306800830FCF79C
S3190000B34C8BFC16490870087800280AD10BE01E22511A0180EF
S3190000B3600830FCF77FFC104908700878002800D05BE702217F
S3190000B3741348FCF781FCF7BDC50700200608002000070020FF
S3190000B38850150020010A0000E40500003AFDFF1F24F2FF1FA9
S3190000B39C0400FA050CED00E0B80400200C050020FC0700208B
S3190000B3B030F2FF1FC0060020A2FDFF1FE4240020E40700206D
S3190000B3C4C80400201B48016801220A430260002019490870EB
S3190000B3D87047F8B50E0017000400174A904208D3164981429E
S3190000B3EC05D3164B984204D3154B834201D30120F2BD8A1AF0
S3190000B400521CBA4201D20220F2BDC019814201D20320F2BDE3
S3190000B414002501E06D1C241DBD4207D2A80031582000F9F735
S3190000B42835FB0028F4D0F2BD0020F2BD000000003C80044070
S3190000B43C010002400000000000000100000400000F0400009B
S3190000B450F2B582B005006F460621F8F7D3FF38802800302136
S3190000B4644143804A55184835B978FE220A402978C909114334
S3190000B478B970B978F9220A40BA707A4AF021490051180191B8
S3190000B48C0121019B1B785B080B4207D090235B008000101818
S3190000B4A0C05A4008084203D0EA781007C00F00E00120E726BD
S3190000B4B4BA783240C0001043019A9278114009010143B9705A
S3190000B4C86846007A012804D00C2818D00D281AD003E0684679
S3190000B4DC00F037F80400E4B220000A38012802D90C380128CA
S3190000B4F014D8A878E72101404000182202400A430820104369
S3190000B50411E0684600F05CF8E8E7684600F058F804000E2C4F
S3190000B518E3D10F24A878E72101404000102210400843A870A4
S3190000B52C28784006400EB978C9010143297068780640B878A3
S3190000B540800018210140314369702000FEBD70B50100F9228E
S3190000B55402230A20012400254D5FDE01B54226D0C026B60030
S3190000B568B54224D07600B5420CD0E026F600B54210D09E0222
S3190000B57CB5420DD090263601B5421CD1022070BD8D78ED08C7
S3190000B590254216D002208C78224007E08D782D0925420ED065
S3190000B5A402208B781A40042313438B7070BD182070BD2E498D
S3190000B5B809780909214200D00B2070BDF1B5012182780A434C
S3190000B5CC82700E20F9230225009E0027F65FFF27BF1CF61BD6
S3190000B5E0022E36D9761F34D0F61E32D0F737F61B31D0B61E4F
S3190000B5F42FD01F4FF61B13D0B61E1CD0F61E0BD0F61E09D040
S3190000B608BF1FF61B1FD0B61E13D0F61E02D0F61E25D023E0A1
S3190000B61CD2080A4220D003E0D00808421CD002200099897851
S3190000B6300B401D4300998D70E6BDD008084211D00098807889
S3190000B644034002201843009988700220E6BD1820E6BD0648AD
S3190000B65800780009084201D01720E6BD1620E6BD30F2FF1F49
S3190000B66C58FBFF1F38FDFF1FFE020000F1B586B019240721BF
S3190000B6806846007EF8F7BEFE694608826846007E302141439F
S3190000B694A24A57184537A249FF22E2328A180392BA79120722
S3190000B6A804D4039A9279D507ED0F00E00025902252008000A7
S3190000B6BC0818801801902B0000AAD21C00880006000F810743
S3190000B6D0890F04A8407800F0B2F806002B0000AA921C0198A8
S3190000B6E400880006000F8107890F6846007C00F0A4F801993F
S3190000B6F809886A4611813A79F92111406A4612891206D20E04
S3190000B70C062313400B433B71F978C909694601D0C97800E0C9
S3190000B7208978039A12786B465A70490006220A4069460A7088
S3190000B734864212D1052E42D0072E09D010243979F9220A40B2
S3190000B7486946097811433971310045E0F9784C06640E072106
S3190000B75C40E0052E01D0052809D13979C906890F012928D16C
S3190000B77003240021002D1FD132E0072E23D0072821D0042ECE
S3190000B78408D1102404213B79F9221A406B461B78134312E0C4
S3190000B7983979C906890F01290FD169464978C90702D4B9792C
S3190000B7AC090708D510240021002D13D03A79F92313403B7163
S3190000B7C00EE005210CE03979F9220A4069460978114339712A
S3190000B7D4072E01D1010000E0310003246A46527852071ED555
S3190000B7E8062E1CD0072E1AD0062818D0072816D03979F92012
S3190000B7FC08406946098909098A0702D10021387108E004225C
S3190000B8108907890F0129114600D1022202433A7110243970B3
S3190000B82408E03970192C05D1132205216846007EF8F732FCBA
S3190000B838200007B0F0BDF1B581B03948009002260124002518
S3190000B84C6846007900283FD010382FD0401F24D0801E2BD051
S3190000B8600A3829D0001F1ED0801E25D00B3823D0C01E18D0F7
S3190000B874801E1FD00C381DD0801E12D0801E19D00938032889
S3190000B88811D9001F14D0401E0DD0801E10D00938052804D9B5
S3190000B89CC01F02D0203817D009E0002916D1002035E00098DC
S3190000B8B000788008204200D0002668460779F0203840103828
S3190000B8C4C7103F0F381800111170002911D123E00720F6BD7B
S3190000B8D8009800780609264201D0042005E0C008204206D0F5
S3190000B8EC0020002B13D1117012E0022E01D105200EE0C1B218
S3190000B900002903D0491E022902D907E0002B03E000990978B5
S3190000B9144908214200D01570C0B2F6BD30F2FF1F58FBFF1F3A
S3190000B9283FFDFF1F38B505000821F8F767FD302169437F4A77
S3190000B93C511849228B5CDF221A404923CA54072489380FD086
S3190000B9507A4BC01A0CD0893804D1202010434931087005E062
S3190000B9640624092203212800F8F796FB200032BDBFB5012400
S3190000B9780025714F785D6946097888422DD0302141436B4A7A
S3190000B98C5118443109782C3907D0491E07D04239012902D948
S3190000B9A0891E02D002E0042400E0032469460979002912D0C7
S3190000B9B4012C10D0902149008200614B9A18515A0A06920F36
S3190000B9C801211140F8F7C0F969460989814200D201246D1CC6
S3190000B9DCEDB2302DCCDB200004B0B0BDF7B590B00026002437
S3190000B9F0002569460E7300270196009610A800783021484388
S3190000BA044C49081846300290008849880918494A1278520082
S3190000BA184B4B9A5A8A4201DA891A00914449C98808188242ED
S3190000BA2C01DA801A0190012104A8FAF779FF302004A90918A5
S3190000BA40491E097810AA1278914227D030225143394A511824
S3190000BA5444310A78202A1BDA3B4A1278D20608D5029A1279B7
S3190000BA689207920F8B799B079B0F9A4212D201226B461A7319
S3190000BA7C019A974202D24A88BF186D1C009A964202D249891E
S3190000BA907618641C401EC0B20028CFD11198047012980570BA
S3190000BAA42C436846007B2043000607D00198874204D30098DF
S3190000BAB8864201D3012000E0002013B0F0BD70B51E4B902207
S3190000BACC520084001C19A2189324A4001C5D802C02D11388AD
S3190000BAE05B045C0F002C24D030235843B04B18183630C67BA2
S3190000BAF45588C27C5207920F0378032B01D10022058A3000C7
S3190000BB08F8F787F9002E05D0761E022E09D9F61E03D00AE03A
S3190000BB1C022C02D103E0032C01D0042C03D1854201DA002065
S3190000BB3070BD012070BD000030F2FF1F77880000000700201A
S3190000BB4458FBFF1FC006002039FDFF1FF3B585B0002569468B
S3190000BB580D809648019096480390934F0078002801D1788911
S3190000BB6C0AE00198407AC00701D5388904E0398978898842B3
S3190000BB8000D30800B989884203D3401A6946488001E068468E
S3190000BB9445806846007D902149008200864B9A1851180291AC
S3190000BBA8302148433C184420205C212819D1029800882100FD
S3190000BBBC44314A79F92111400206D20E062313400B432100F9
S3190000BBD044314B710009800703D1210044314D7003E004206C
S3190000BBE42100443148704420205C20380F2842D220004430E2
S3190000BBF800794006400E032801D1002600E00126310068461D
S3190000BC0C007DFFF75AFF002800D199E00198C078C00909D06D
S3190000BC20388B800506D50220243420700B200699087096E025
S3190000BC3420002430807C032875D031006846007DF8F784F84F
S3190000BC482100443148806846428801980078019949794B084C
S3190000BC5C0340D907C90F6846007DFFF785FE242160541526FB
S3190000BC70C01E012804D8069806704434658070E03878000165
S3190000BC844D490818C1880A290FD103984078802803D102982B
S3190000BC9800880005800F032801D1029801E0200044304088A2
S3190000BCAC00E0084669464988814238D2388B80214900014312
S3190000BCC0398301980078C00731D46A4600A9491C6846007DE8
S3190000BCD4FFF788FE002828D00198007A000722D5F88869467A
S3190000BCE849786A461278914200D37888443461884418387834
S3190000BCFC40003049085AA4B2A04210D2241A68464078904283
S3190000BD1008D304210D20F8F7FBFA81B2A0B2FDF7DCFD02E0D4
S3190000BD24A0B2FBF776F801201AE006980670200044304580CB
S3190000BD3803980078002801D1042000E00320243420700AE0EB
S3190000BD4C0520242160540C200699087020002430807C0328E1
S3190000BD608BD1002007B0F0BD30214843104909180800443017
S3190000BD747F2203791340032B06D10078212801D106200DE09A
S3190000BD8805200BE003791A40042A01D1072005E000782128EE
S3190000BD9C01D1122000E01120012224310A7006490A71704705
S3190000BDB030F2FF1F38FDFF1FA2FDFF1F58FBFF1FC0060020D2
S3190000BDC4E4070020FEB5040000206946087103212000F8F728
S3190000BDD89BFA6C216143A64A5118B13100910D78A44909192B
S3190000BDECA44A02920222FD23AE070AD5029FBE5EB04212DA48
S3190000BE001D40009E35700D78FE262E400AE0029E0027F65F6B
S3190000BE14864206DA1543009E35700D7801262E430E70974D52
S3190000BE286400AE4E3419645B009D2D780E78844208DA012300
S3190000BE3C6F463B712B43009D2B7032430A7005E0FE222A4087
S3190000BE50009D2A7033400B70C830A04202DA002069460871B5
S3190000BE6468460079FEBDF8B5002400250126814F9C48385A7F
S3190000BE780121A940084213D0E8B2FFF7A1FF204304006C2055
S3190000BE8C68433818B13000784008304206D006220321280044
S3190000BEA07F38C0B2F8F7FAF86D1C0C2DE2DB8F4820212406BD
S3190000BEB401D00160F1BD4160F1BDF8B504210D20F8F724FA39
S3190000BEC880B289490A781201844B9A1856889288864B1C78E9
S3190000BEDC64001C705C7864005C70202401250F8BBF082F421C
S3190000BEF00ED00A3EB0421E7803DB012737431F7017E0002E56
S3190000BF0415D10E8B7B4F37400F8310E086420EDA1F78012673
S3190000BF183E431E70FF2E08D10E8B042737430F83744E3668CA
S3190000BF2C7778274377700E8B2E420CD00A328242587802DB29
S3190000BF4005435D70F1BD002812D16D4830400883F1BD9042E9
S3190000BF540CDA5A78012010435870FF2806D135430D8365482C
S3190000BF68006841780C434470F1BD644908884000634A126849
S3190000BF7C5206D30F01225A401043088059490A8BD30604D5F0
S3190000BF90000409D15D48104005E080B25C4B984202D1102029
S3190000BFA4104308837047FCB54D4C5948201800904E4D007828
S3190000BFB8002801D16E8800E0EE8828780001275A0098807F70
S3190000BFCC0A214843391A0020012900DA0021009AD27F0A23F5
S3190000BFE05A43BA1A012A00DB1000864203D2A87BFB220240A1
S3190000BFF4AA738E4203D3A87B04210143A9730098007F7843F6
S3190000C0086421F8F7A6FB01900098407F474338006421F8F7EB
S3190000C01C9EFB864203D2A87BFD210140A9730198864203D3FF
S3190000C030A87B02210143A9730120F4214900615C4907490F6C
S3190000C044022902D0042906D00FE0298B314A0A40A97B490805
S3190000C05804E0298B2E4A0A40A97B89080840C00110432883B8
S3190000C06CF3BD288B294901402983F3BD5015002004F2FF1FAF
S3190000C080781800004E020000F8B500240125234E1548305A77
S3190000C0940121A140084210D06C2060433718B1373878400807
S3190000C0A8284202D02802FAF7B7FC3878284202D06802FAF72D
S3190000C0BCB1FC641C0C2CE5DB0A4C208B000A284202D02803D3
S3190000C0D0FAF7A6FC207E0521084202D06803FAF79FFCF1BD3E
S3190000C0E458FBFF1FE4050000C4F00F4030F2FF1FDA070020A4
S3190000C0F8FBFF000024F2FF1FFEFF00002CF2FF1FD0F00F40B8
S3190000C10CEFFF0000FFFF00004A0200007FFF000050150020DE
S3190000C12080B5FFF7CCFEFFF724FFFFF79EFEFFF7ABFFFFF7CF
S3190000C1343AFF01BD10B5040009220321F7F7ACFF00203021D8
S3190000C1484C43454909192431087010BD38B50500F0240221DB
S3190000C15CF8F752F9002810D109212800F8F74CF9002809D0FF
S3190000C170302045433A48401944300078762802D0762400E02C
S3190000C1845024200032BD38B5354D0124287A002807D01B22AC
S3190000C19803218020F7F77EFF002028720BE0687A002808D1D6
S3190000C1ACA87A002805D01B2204218020F7F770FF6C7228886D
S3190000C1C04109000920420AD0214213D11A2203218020F7F7A1
S3190000C1D463FF28882021014309E0214208D01A220421802095
S3190000C1E8F7F758FF28881E49014029802888C1088008204294
S3190000C1FC0AD0214213D1182203218020F7F748FF28880821FC
S3190000C210014309E0214208D0182204218020F7F73DFF2888D3
S3190000C2241149014029802888410820420AD0214213D1192205
S3190000C23803218020F7F72EFF28880221014309E0214208D0D2
S3190000C24C192204218020F7F723FF2888B2490140298031BD45
S3190000C26030F2FF1F48F2FF1FDFFF0000F7FF0000F2B582B07F
S3190000C27430214143AB4A511800910C46403425790126617A86
S3190000C288890931420FD0A17A490931420BD100220721F7F7C4
S3190000C29CFFFE607A4006400E6072FBF758FC206046E00299C4
S3190000C2B0490B314001D05620FEBD02A9C978314204D0FBF788
S3190000C2C44AFC20607220FEBD4A08324204D0FBF742FC206003
S3190000C2D87320FEBD029A9209324005D0102D01DB6120FEBD2B
S3190000C2EC6E20FEBD8A08324204D0FBF730FC20607420FEBD28
S3190000C300C908314201D07720FEBDAF4F029900290BD10521F8
S3190000C314F8F776F8002864D1102D65DAB87820210143B970FB
S3190000C32808E0072D02DAFBF714FC206002984009304001D05D
S3190000C33C7520FEBD0298000D304001D07820FEBD009839305B
S3190000C3500299890A31400AD04178FF2901D0491C4170102D55
S3190000C36401DB5920FEBD6420FEBD0299490C31400AD041787C
S3190000C378FF2901D0491C4170102D01DB5A20FEBD6520FEBD0E
S3190000C38C0299C909314006D00178FF2901D0491C01706F200C
S3190000C3A0FEBD0299090A314006D00178FF2901D0491C01708B
S3190000C3B47120FEBD0299490A314012D10299890B31400ED162
S3190000C3C80299C90C31400AD10299090B314006D10299490DB7
S3190000C3DC314002D10299890C314000D09AE0202D00DB97E079
S3190000C3F00221029A120932400FD0C278FF2A01D0521CC27034
S3190000C404102D01DB5E20FEBDE07A304201D00143E1726A200E
S3190000C418FEBD029A324015D08278FF2A01D0521C8270102DCB
S3190000C42C01DB5C20FEBDE07A304201D00143E172607A40098C
S3190000C440304201D06820FEBD6620FEBD029A920832400BD098
S3190000C4540278FF2A01D0521C0270E07A304201D00143E17246
S3190000C4687020FEBD029AD20832400FD04278FF2A01D0521C86
S3190000C47C4270102D01DB5820FEBDE07A304201D00143E17274
S3190000C4906320FEBD029AD20B324015D08278FF2A01D0521C22
S3190000C4A48270102D01DB5D20FEBDE07A304201D00143E17207
S3190000C4B8607A4009304201D06920FEBD6720FEBD029A120CC4
S3190000C4CC32400FD0C278FF2A01D0521CC270102D01DB5F2099
S3190000C4E0FEBDE07A304201D00143E1726B20FEBD029A520817
S3190000C4F432400FD0C278FF2A01D0521CC270102D01DB602070
S3190000C508FEBDE07A304201D00143E1726C20FEBDB878802112
S3190000C51C0143B970F020FEBDFDFF000030F2FF1F7CB501005F
S3190000C53030224A43954B9A184423D45C02232500052D0ED986
S3190000C544203D012D28D9213D37D00F3D35D06D1E042D21D9E5
S3190000C558233D30D0ED1E1DD028E04923D55CC026354207D098
S3190000C56C79246906490EAB09DB010B4349321FE090256D00D8
S3190000C5808900834E7118495BC90B01D1792416E04B20105C0A
S3190000C59401434B32117012E090256D0089007B4E7118495BB8
S3190000C5A8C90B03D04921515CC90904D04B21515C0B434B3231
S3190000C5BC1370FFF7BBFD200076BD0000E424002030214843DD
S3190000C5D06E4908184421415C012902D9C91E022907D84B2116
S3190000C5E4415CCA0703D5FE220A404B3002707047F1B584B00F
S3190000C5F8FBF7AFFA69460E7C624C302171436718403739680B
S3190000C60CFBF7A8FA01000125F87A400828420FD03879742809
S3190000C62008D090204000B200594B9A18105A284200D084E028
S3190000C634F87AFD220240FA725548007840080122024068463D
S3190000C6480272183400942388514881428041C043C00F019059
S3190000C65C4F4C0020FA22D2003E79103E042E60D9103E2ED05F
S3190000C670213E2CD0103E012E29D9B61E54D0761E012E3DD905
S3190000C684B61E012E3FD9B61E0A2E4BD90B3E022E2AD9F61EC1
S3190000C698012E1BD9B61E012E1ED9B61E022E3FD9F61E34D037
S3190000C6AC761E25D0761E022E45D9F61E4AD0761E4CD0761E97
S3190000C6C04ED0761E04D0B61E51D0761E2CD05AE0914217E051
S3190000C6D46A46127A002A0FD02E4A24E06A46127A002A2CD128
S3190000C6E8A1420BE05208294B1B789B082B4218D1914203E05A
S3190000C6FC019843E0600881428041C0430CE0580A0121414088
S3190000C7100D40280038E003216846007CF7F772FE401E8041B7
S3190000C724C00F2FE0920091420AE09008814204D300210B2050
S3190000C738F8F7E6FB23E0002022E0A14220D31648807900289D
S3190000C74C1CD01AE0914219D3590706E0914215D3D90702E06B
S3190000C760914211D3D906C90F012048400CE01100009840686B
S3190000C774FBF7FDF9002801D0009885720098807A00E00120A8
S3190000C78805B0F0BD30F2FF1F58FBFF1F76180000EE02000006
S3190000C79C88130000E4070020F3B583B06846007B02903021F6
S3190000C7B0484399490E18370044373878694608716846047927
S3190000C7C4007BFFF715FF002801D1F020B8E105216846007BE4
S3190000C7D8F7F714FE002811D06846007941280DD18C48007884
S3190000C7EC002809D08B48817840220A4382706846007BFFF7A6
S3190000C8009BFC94E124369020400002998900854A511808184C
S3190000C81400900220002569460979103900D148E1491E00D187
S3190000C82847E1491E00D148E1491E00D147E1491E00D140E1B4
S3190000C83C0C3904D0491E00D1D8E0491E0C2900D870E01F39BD
S3190000C8505FD0103954D0491E03D0491E01294FD9891E00D1C7
S3190000C86431E1491E012949D9891E16D0491E17D0491E18D0CB
S3190000C878491E00D129E1491E1AD0491E1BD0491E1CD0491E07
S3190000C88C1DD0491E1ED0491E34D0491E00D12AE1491E00D16A
S3190000C8A015E1491E00D116E1491E00D115E1491E02D0491E8B
S3190000C8B403D0491E00D110E1491E00D10FE1491E00D10EE11F
S3190000C8C8491E00D10DE1491E00D10CE1491E13D0491E11D079
S3190000C8DC491E012900D808E1891E00D107E1491E022907D91E
S3190000C8F0C91E00D11AE1491E00D100E1491E012900D807E111
S3190000C904891E00D106E1491E00D108E10DE104980105C90F31
S3190000C91801D0562012E100980078C00700D52024B879800624
S3190000C92C03D408E1B879800601D52124F9E07F207979C90923
S3190000C94005D0B979890602D4797901407971334949780029EE
S3190000C95450D03A7902400A3A012A07D90C3A012A18D9921E53
S3190000C96845D0521E35D043E0327DFF2A01D0521C32755124D5
S3190000C97C397908400B2800D15224B5490978890734D554249D
S3190000C9900B2831D155242FE0327DFF2A01D0521C327551249D
S3190000C9A439790840172800D1522400980088400620D5F52089
S3190000C9B8400002994900194A511808180178FF2916D0407816
S3190000C9CCFF2813D03879C00910D154240EE0707EFF2801D0A0
S3190000C9E0401C707653240023532239786846007BFAF72CF8FD
S3190000C9F400E020240848C07801285BD13078022823D019D377
S3190000CA08042838D02CD306280AD036D312E000BF30F2FF1FDF
S3190000CA1CE4070020E424002058FBFF1F35706224FBF795F8B2
S3190000CA30F061B07DFF2801D0401CB07500980078C00774D4D6
S3190000CA44B879800671D4412479E09D48008B8005F2D55724E7
S3190000CA580023224639786846007BF9F7F3FFE9E77124357073
S3190000CA6CFBF775F8F061707DFF28EFD0401C7075ECE76F2486
S3190000CA80F3E75B243570FBF768F8F06100235B2239786846FC
S3190000CA94007BF9F7D9FF707DFF2801D0401C7075B879800668
S3190000CAA8C8D578798021014379715B2046E0002439E0012414
S3190000CABC37E0052435E0022433E0032431E02E242FE02224F3
S3190000CAD02DE025242BE0232429E0242427E0262425E02724B2
S3190000CAE423E0282421E029241FE02A241DE02B241BE02C24B7
S3190000CAF819E02D2417E002216846007BF7F77EFC002810D027
S3190000CB0C30213000FAF78EF820240AE07A24F9790843F87125
S3190000CB2005E0F02400980078C00700D44124B879800606D560
S3190000CB347879C00903D03878792800D00400200005B0F0BDB3
S3190000CB48F1B582B06846007A302141435B4A571844373978BE
S3190000CB5C6A461171F52149004000584A1018405CFF2801D18F
S3190000CB705020FEBD6846007AFFF7ECFA04007F260125F02895
S3190000CB842AD16846007AF7F735FD009001466846007AFFF75F
S3190000CB986BFB0400F02C03D06846007984420ED16846007A36
S3190000CBACFFF70EFD00996846007AFFF7F5FD0400F02C2FD1A5
S3190000CBC0684604792CE0B8794009284224D07879064080098C
S3190000CBD4C001304378711DE0B9794909294219D079797F22C2
S3190000CBE80A408909C90111437971742810D1002207216846DA
S3190000CBFC007AF7F74DFA787906407E71B879DF210140B971AE
S3190000CC107879FE21014079716846007AFFF78CFA2A48007841
S3190000CC24032804D16846007AFFF77EFC04002000FEBD10B5BA
S3190000CC38002030214143214A511849314A78DF2313400A7806
S3190000CC4CD407A20E1A434A70401C3028EFDB10BD3AFDFF1F8C
S3190000CC60F8B51B480078002801D0FFF7E4FFFFF78CFA0027BD
S3190000CC7400241748005D00903021484310490E1844363578B4
S3190000CC880098FFF75DFF3070202D06DA202804DB0F480078E5
S3190000CC9C400600D477800123327829000098C0B2F9F7CEFEB0
S3190000CCB0641C302CDFDB06484078002801D004484770F1BD24
S3190000CCC430F2FF1F58FBFF1F19050020E40700200007002035
S3190000CCD83DFDFF1FF8B500270026302070431C490C184434EC
S3190000CCEC207820282BDA0121F0B2F7F785FB050004210D20C0
S3190000CD00F7F706FB80B26843FA218900F7F725FD6081012097
S3190000CD14114909784909014217D061890F4A1288891AF42218
S3190000CD289200914204DB217B49000843207300E02773207BD5
S3190000CD3CFF2806D111220321F0B2F7F7A9F967812773761C42
S3190000CD50302EC6DBF1BD00BF30F2FF1F40FDFF1F5CFCFF1F4C
S3190000CD64F0B58DB0002201218020F7F795F9012101A8F9F7B8
S3190000CD78D9FD0025194F68001949085A7988884224D2081A2F
S3190000CD8C69460880302401A80019401E0078302141437E18FF
S3190000CDA044363178202911DA2A000221F7F776F970896946D0
S3190000CDB40988884203D300206946088008E069460988081A93
S3190000CDC869460880641EE4B2002CDED16D1C102DD1DB012094
S3190000CDDC034908700DB0F0BD30F2FF1FC006002006080020BB
S3190000CDF0F8B50400F7F7D2FF674A00216748F7F7C3FEFCF796
S3190000CE04DDFD012C01D0F7F7FDFC00200021634D0A01634BAB
S3190000CE189A5A4B00EB181A851A81491C1029F5DB002180274E
S3190000CE2C30224A435A4B9A181300443350261E701E793E4013
S3190000CE401E7124321070491C3029EFDBF6F7FAFB0126554845
S3190000CE5400788009304201D153490E705348688053498E7147
S3190000CE68FEF762F952480078082802D1FCF778FF05E0FAF70B
S3190000CE7C6EFE4749C8614E480670002C03D100210120F5F73D
S3190000CE9041FFF1BDF0B583B0062200216846F7F773FE474CD9
S3190000CEA400272770464D2888002802D0FCF7CAF80AE069462B
S3190000CEB8FAF75EF8684600882880002802D00020FFF792FF9A
S3190000CECC2078012804D020D3032818D00CD31CE0F8F74CFAA1
S3190000CEE00E2203218020F7F7D9F82888002807D0012003E0D2
S3190000CEF42888002802D00220FFF778FF002131A0F5F7F6FE19
S3190000CF0805E0FFF7A9FEF8F733FAFCF7D1FE27700126607819
S3190000CF1C4008304202D0072024490870F9F7C5FBF9F788FE3D
S3190000CF30607840083042C9D1B7E770B5FDF733FC002827D0B6
S3190000CF4421480068C17802220A43C270124C114A002120002C
S3190000CF58F7F716FE1C4A00211C48F7F711FE002000218026EE
S3190000CF6C30224A43A2181300443350251D701D7935401D71ED
S3190000CF8024321070491C3029F0DBF9F794FBF9F757FEFAE793
S3190000CF9470BD00002409000030F2FF1FB806002058FBFF1F9A
S3190000CFA83DFDFF1F02080020FF7F0000E407002054FBFF1FF7
S3190000CFBC50F2FF1F19050020341B00202577000024F2FF1F7E
S3190000CFD0040A00005015002080B55B4800F012F800F017F8E3
S3190000CFE400F036F858485949416007210160F9F721FEF9F7AA
S3190000CFF851FFFDF7B7FBFEF7E3F901BD5349014053480160C1
S3190000D00CBFF34F8F704752490020086348638863C86380223A
S3190000D020D2040A60C860920A0A644D4906220A704870A022D2
S3190000D034CA70087148718879C006FCD588790C221042FBD191
S3190000D048464800E000BF401EFCD17047F82080014349086032
S3190000D05C434944480860486043480864434A4A648A64CA6444
S3190000D07080235B048B6741490A604A60C860486488643F49CC
S3190000D0840A604A603E4A136053609060D0603D4910234B6745
S3190000D0981061506190613B4A1060506090604030D06008200E
S3190000D0AC0867384802689A43026020220A6740230B678023A7
S3190000D0C00B6742630363D202026704220A6000220A64E82173
S3190000D0D40160A02101642E482E490860704730B52D480278DB
S3190000D0E840782D4980231A4206D00C68002525600C682578FC
S3190000D0FC2B43237020231A4203D00C6825782B432370402332
S3190000D1101A4003D00A681478234313700422104204D00B6832
S3190000D1249C78102525439D700823184203D00C6825782A435D
S3190000D1382270800703D5086801780B43037030BD0014000041
S3190000D14C10E000E063BB000000FFFF3F08ED00E00480044001
S3190000D16000400640B25D00003880044000D00440000300010C
S3190000D17400010001000200010490044000A0044004B00440E8
S3190000D18814F00F4010C0044094F00F400100070014F10F40F7
S3190000D19C00F0074024F2FF1F00B5012012490968002907D567
S3190000D1B010490968802212060A430E490A600AE00D49096822
S3190000D1C4497804220A430B4909684A70C0B20028FCD100BD7A
S3190000D1D800B5012006490968097810220A43044909680A706F
S3190000D1ECC0B20028FCD100BD2CED00E024F2FF1F80B5FFF7AD
S3190000D200D1FF01BD80B5FFF7E7FF01BD80B5FFF7C9FF01BD06
S3190000D21480B5FFF7C5FF01BD80B5FFF7C1FF01BD80B5FFF77F
S3190000D228BDFF01BD80B5FFF7B9FF01BD80B5FFF7B5FF01BD34
S3190000D23C80B5FFF7B1FF01BD80B5FFF7ADFF01BD80B5FFF77F
S3190000D250A9FF01BD80B5FFF7A5FF01BD80B5FFF7A1FF01BD48
S3190000D26480B5FFF79DFF01BD80B5FFF799FF01BD80B5FFF77F
S3190000D27895FF01BD80B5FFF791FF01BD80B5FFF78DFF01BD5C
S3190000D28C80B5FFF789FF01BD80B5FFF785FF01BD80B5FFF77F
S3190000D2A081FF01BD80B5FFF77DFF01BD80B5FFF779FF01BD70
S3190000D2B480B5FFF775FF01BD80B5FFF771FF01BD80B5FFF77F
S3190000D2C86DFF01BD80B5FFF769FF01BD80B5FFF765FF01BD84
S3190000D2DC80B5FFF761FF01BD80B5FFF75DFF01BD10B5F9F7F5
S3190000D2F0A5F8194C194AFF212000F7F745FC1848201880F345
S3190000D3040988022080F31488FFF764FEFFF7E7FEFCF796FC95
S3190000D318F9F7A0F8F9F76BFAF9F78EFCF9F792F8FFF707FE2F
S3190000D32C0D490E480068FAF77FFC0020FFF75AFDF9F76FFAA1
S3190000D340FCF77BFF032200210848F7F71DFCFFF7A1FD002015
S3190000D35410BD00BF08080020480D0000440D0000416C0000B0
S3190000D368DC180000E42400202563256325632563256325635F
S3190000D37C256325632563256300000000256325632563256357
S3190000D39025632563256325632563000025772577256300001B
S3190000D3A42577257725772563257700002563257725530000DB
S3190000D3B8256325770000000025632553000000002563256327
S3190000D3CC256325632563256325632563000000004F637420D1
S3190000D3E03137203230313700000000000000000000000000E1
S3190000D3F400000000000031373A31393A34370000000000006E
S3190000D408000000000000000000000000000000004E6565648E
S3190000D41C20746F2066696C6C0000000038B401210268001D97
S3190000D430002A0FD00368C318446808300C4202D04D466D1E71
S3190000D44464191D6825601B1D241D121FECD0F8E732BC70475D
S3190000D45801000000280000003A1500002B15000018D4000016
S3190000D46CC8170000CC170000CD170000CA170000CE1700003A
S3190000D48010B5074979441831064C7C44163404E0081D0A68A0
S3190000D494891888470100A142F8D110BD080000002800000064
S3190000D4A87361FFFFD815000030F2FF1F0000000071FFFFFFFD
S3190000D4BC200200006400000010F0FF1F0000000000F00BF8BF
S3190000D4D0002801D0FFF7D4FF0020C046C046FFF705FF00F06A
S3190000D4E402F80120704780B500F002F801BD000007463846B4
S3190000D4F800F002F8FBE7000080B5C046C046024A1100182078
S3190000D50CABBEFBE726000200C046C046C046C046FFF7D6FFAF
S3190000D52058D4000004E045490978090603D4401E0028F8D19D
S3190000D534704701207047F8B5040000F08FF801253E4FFA2059
S3190000D5480001FFF7EBFF002803D1387805433D7033E0384EAE
S3190000D55C702030700920F071200CB071200A70713471307856
S3190000D5708021014331703348FFF7D4FF002802D13878022109
S3190000D5841BE03078712108421ED170203070F571200CB0713C
S3190000D598200A70713471F5720020B0727072307880210143B1
S3190000D5AC3170FA200001FFF7B7FF002804D1387804210143E7
S3190000D5C0397041E030787121084200D040E043E0F8B504003F
S3190000D5D40F0000F043F8194DFA200001FFF7A0FF002802D1F2
S3190000D5E8287801211CE0134E702030700620F071200CB07106
S3190000D5FC200A70713471380EF072380CB072380A707237728A
S3190000D6103078802101433170FA200001FFF782FF002804D143
S3190000D62428780821014329700CE030787121084200D00BE01B
S3190000D6380EE0000000000240E424002080841E0000F012F864
S3190000D64C0520F2BD00F00EF80420F2BD00F00AF80020F2BD66
S3190000D66008480178002900D172B6491C017070470448017873
S3190000D674002903D0491E0170090600D162B6704701080020F0
S3190000D688540400200100640000006300000000000000000048
S3190000D69C000000000000000000000000000000000000000074
S3190000D6B034050020010064000000630000000000000000003F
S3190000D6C400000000000000000000000000000000000000004C
S3190000D6D8000000000000010000000000000000000000000037
S3190000D6EC000000000000000000000000000100000000000023
S3190000D70000000000000000000000000000000000000000000F
S3190000D7140000FF0000000000000000000000000000000000FC
S3190000D72800000000FFFF000000900100FC9F010004F0FF1FAA
S3190000D73CC0000000FFFF0000FAFAFAFAFAFAFAFAFAFAFAFA5D
S3190000D750FAFAFAFAFAFAFAFAFAFAFAFAFAFAFAFAFAFAFAFA37
S3190000D764FAFAFAFAFAFAFAFAFAFAFAFAFAFAFAFAFAFAFAFA23
S3190000D778FAFAFAFAFAFAFAFAFAFAFAFAFAFAFAFAFAFAFAFA0F
S3190000D78CFAFAFAFAFAFAFAFAFAFAFAFAFAFAFAFAFAFAFAFAFB
S3090000F3FC0C68DC1E99
S70500000000FA
